:1000000002407E124EF112541280FB02446FE490C3
:100010000266F0EF5407F022D2B422024EAF75E12F
:100020003F22320245E653A67F43890130220875FC
:100030008CE5758AF68011302108758CE0758AC0D0
:100040008006758CF0758A6043B802D2A9D28C22E2
:10005000C2B422024D51302303D2B522D2B2224380
:10006000E7202202383530211378E07C017D017BC6
:10007000017A0179F77E007F11120E27301979C2BB
:10008000199001E1E0FF30E709D22AE4900368F01B
:100090008006900368E004F0900368E0C394054094
:1000A000057405F0C22A202A4F90036FE06F543088
:1000B0006002D2289001E2E0FF90036DE06F700CC7
:1000C0009001E3E0FE90036EE06E6002D22B90019F
:1000D000F0E030E504D22E8002C22E9001E0E090E4
:1000E0000371F09001E1E090036FF090036DEFF089
:1000F0009001E3E090036EF0222222020022E490BD
:1001000002F7F0A3F0A3F078007C037D017BFF7A77
:10011000737920FE7F12120E2730230F9002F8749D
:1001200001F0A37406F012424C8015E49002F830FE
:10013000210AF0A37403F01243ED8004F0A304F04D
:10014000900294E09002FEF0900295E09002FFF0A1
:100150009002FAE590F0A3E5A0F0A3E5B0F0A3E5E6
:10016000E8F09002F8E09002F7F09002F9E0FF90DA
:1001700002F7E0FEC39F400302065FEE75F008A49D
:100180002490F582E43472F583E493607C9002F766
:10019000E0FF75F003A42400F582E43403F583E066
:1001A000FBA3E0FAA3E0F9120E4D5401FEEF75F047
:1001B00008A424C0F582E43472F583E4936EFD90C4
:1001C00002F7E075F008A42496F9740235F0FA7B82
:1001D00001E075F008A424F0F582E43472F583E4BC
:1001E00093900390F0747F2FF582E43402F583E05E
:1001F000124E2BEF5401FF9002F7E0247FF582E4CA
:100200003402F583E054FE4FF09002F7E0FE75F003
:1002100008A42491F582E43472F583E49370030218
:1002200002A49002F7E0FF75F003A42400F582E435
:100230003403F583E0FBA3E0FAA3E0F9120E4DC30B
:10024000135401FDEF75F008A424C1F582E4347263
:10025000F583E4936DFDEE75F008A42497F974021C
:1002600035F0FA7B019002F7E0FF75F008A424F165
:10027000F582E43472F583E493900390F0747F2F59
:10028000F582E43402F583E0C3124E2AEF540125CF
:10029000E0FF9002F7E0247FF582E43402F583E08A
:1002A00054FD4FF09002F7E0FE75F008A42492F59B
:1002B00082E43472F583E49370030203409002F702
:1002C000E0FF75F003A42400F582E43403F583E035
:1002D000FBA3E0FAA3E0F9120E4D13135401FDEF56
:1002E00075F008A424C2F582E43472F583E4936DBA
:1002F000FDEE75F008A42498F9740235F0FA7B013C
:100300009002F7E0FF75F008A424F2F582E434725D
:10031000F583E493900390F0747F2FF582E4340228
:10032000F583E0124E29EF540125E025E0FF90020D
:10033000F7E0247FF582E43402F583E054FB4FF0CC
:100340009002F7E0FE75F008A42493F582E434727D
:10035000F583E49370030203DE9002F7E0FF75F08B
:1003600003A42400F582E43403F583E0FBA3E0FA60
:10037000A3E0F9120E4D1313135401FDEF75F008AD
:10038000A424C3F582E43472F583E4936DFDEE7525
:10039000F008A42499F9740235F0FA7B019002F771
:1003A000E0FF75F008A424F3F582E43472F583E4E9
:1003B00093900390F0747F2FF582E43402F583E08C
:1003C000124E28EF540133333354F8FF9002F7E014
:1003D000247FF582E43402F583E054F74FF0900275
:1003E000F7E0FE75F008A42494F582E43472F583F6
:1003F000E49370030204799002F7E0FF75F003A420
:100400002400F582E43403F583E0FBA3E0FAA3E0E3
:10041000F9120E4DC45401FDEF75F008A424C4F583
:1004200082E43472F583E4936DFDEE75F008A42444
:100430009AF9740235F0FA7B019002F7E0FF75F04B
:1004400008A424F4F582E43472F583E493900390D5
:10045000F0747F2FF582E43402F583E0C4124E2B52
:10046000EF5401C454F0FF9002F7E0247FF582E4DA
:100470003402F583E054EF4FF09002F7E0FE75F0A0
:1004800008A42495F582E43472F583E493700302A2
:1004900005169002F7E0FF75F003A42400F582E44E
:1004A0003403F583E0FBA3E0FAA3E0F9120E4DC498
:1004B000135401FDEF75F008A424C5F582E43472ED
:1004C000F583E4936DFDEE75F008A4249BF97402A6
:1004D00035F0FA7B019002F7E0FF75F008A424F5EF
:1004E000F582E43472F583E493900390F0747F2FE7
:1004F000F582E43402F583E0C4124E2AEF5401C4BD
:100500003354E0FF9002F7E0247FF582E43402F5F3
:1005100083E054DF4FF09002F7E0FE75F008A4246A
:1005200096F582E43472F583E49370030205B59086
:1005300002F7E0FF75F003A42400F582E43403F52C
:1005400083E0FBA3E0FAA3E0F9120E4DC4131354A9
:1005500001FDEF75F008A424C6F582E43472F5833A
:10056000E4936DFDEE75F008A4249CF9740235F057
:10057000FA7B019002F7E0FF75F008A424F6F582FB
:10058000E43472F583E493900390F0747F2FF58246
:10059000E43402F583E0C4124E29EF5401C433332E
:1005A00054C0FF9002F7E0247FF582E43402F58323
:1005B000E054BF4FF09002F7E0FE75F008A42497D6
:1005C000F582E43472F583E49370030206569002D8
:1005D000F7E0FF75F003A42400F582E43403F5830B
:1005E000E0FBA3E0FAA3E0F9120E4DC41313135479
:1005F00001FDEF75F008A424C7F582E43472F58399
:10060000E4936DFDEE75F008A4249DF9740235F0B5
:10061000FA7B019002F7E0FF75F008A424F7F58259
:10062000E43472F583E493900390F0747F2FF582A5
:10063000E43402F583E0C4124E28EF5401C433338E
:10064000335480FF9002F7E0247FF582E43402F512
:1006500083E0547F4FF09002F7E004F002016A203B
:100660002303302110900280E09001AAF0900281D3
:10067000E09001ABF0202303020738E4900312F06E
:10068000900283E0FC5408131313541FFE900312CE
:10069000E054FE4EF0EC5404C313FFE054FD4FF061
:1006A000900284E05408C313FF900312E054FB4F00
:1006B000F0900282E0FC5480C4540FFE900312E0DC
:1006C00054F74EF0EC54401313543FFFE054EF4FF7
:1006D000F0900282E0FC5420FE900312E054DF4EC2
:1006E000F0301F17EC541025E025E0FFE054BF4F19
:1006F000F0EC5402C4333354C0801D900282E0FCFD
:100700005402C43354E0FE900312E054BF4EF0ECA8
:100710005401C43333335480FFE0547F4FF09003CF
:1007200012E090028BF0E0FF123DCE90028BE030A1
:10073000E603D21D22C21D2230212990027FE0FF54
:10074000900289F0123DCE900289E020E40312006D
:100750005F900289E054C0FFBFC004D21D8002C276
:100760001DEF804E30225390027FE090028AF030DD
:100770002506E030E302800A30240A90028AE02055
:10078000E30312005F301E0B90028AE054287003CE
:1007900012005F90028AE030E40312005F90028A48
:1007A000E0FF54C0FEBEC004EF543FF090028AE068
:1007B00054C01313543F90027EF022C123C11FC1C5
:1007C00020C121C122C125C124C11EC11D6030022A
:1007D0009600000000000000000000000000000083
:1007E0000000000000000000000000000000000009
:1007F00000000000000000000000000000000000F9
:10080000004A028C000000000000000000004102CD
:100810008B004102890041028A0041027E00C13EF4
:10082000C13D44026D000000004101D00001720092
:10083000017100175A0000000000000000000000D5
:100840000000000000000000000000000174000132
:100850007300187D00000000000000000000000090
:1008600000000000000000000000000041026C00D9
:1008700041026B0057023C00000000000000000035
:100880000000000000000000000000000000410126
:10089000DF004101DE004D01D1000000000000003A
:1008A0000000000000005701F700000000000000F9
:1008B0000000000000000000000000000000000038
:1008C0005701E000000000000000000000000000F0
:1008D000000000000000000000005802530000006B
:1008E0000000000000000000000000000000000008
:1008F000000000000057022500000000000000007A
:100900000000000000000000000000000000005790
:10091000020E0000000000000000000000000000C7
:100920000000000000000000004D02710000000007
:1009300000000000000000000042039D0000420390
:100940009F0000C13F420104000042010600006117
:100950000400000000000000000000000000000093
:100960000000000000000000000000000000000087
:100970000000000000000000000000000000000077
:100980000000000000000000000000000000000067
:100990000000000000000000000000000000000057
:1009A0000000000000000000000000000000000047
:1009B0000000000000000000000000000000000037
:1009C0000000000000000000000000000000000027
:1009D0000000000000000000000000000000000017
:1009E0000000000000000000000000000000000007
:1009F00000000000000000000000000000000000F7
:100A000000000000000000000000000000000000E6
:100A100000000000000000000000000000000000D6
:100A200000000000000000000000000000000000C6
:100A300000000000000000000000000000000000B6
:100A400000000000000000000000000000000000A6
:100A500000000000000000011B00011A0001090055
:100A6000010800580313FF542BFF5348FF5272FF35
:100A70005419FF541FFF00F9FF00FAFF5434C13C22
:100A80004103B5004103B300C138C139C13AC13B8C
:100A90004103B400C119C114C115C11AC11CC1164A
:100AA000C117C113C118C11B017500017600017780
:100AB000FF0179FF0178FF017AFF019900019A0097
:100AC0000195FF0197FF0196FF0198FF4103720016
:100AD000410376004103770041037A00410373002C
:100AE000410379004103740041037500410378001C
:100AF000C108C10DC10CC107C105C109C111C104A3
:100B0000C10FC10AC110C10BC106C10EC112410102
:100B10009C004101A8004101A9004101CA00440113
:100B2000B0000000004401BF000000004101CB0004
:100B30004101A7004101C60041019A014101CE00D7
:100B40004101C7014101B5004101BE004201C80099
:100B50000041019B004101C5004101C3004101B4B6
:100B6000004801B600000000000000004101AE0096
:100B70004101A6004101CC004101CD004101CF005F
:100B800049019D0000000000000000004101AF008D
:100B90004101C4004101AA004101AB00C100C101F3
:100BA000C102C103410108004101090041010A00DD
:100BB0006080010B00000000000000000000000049
:100BC0000000000000000000000000000000000025
:100BD0000000000000000000000000000000000015
:100BE0000000000000000000000000000000000005
:100BF00000000000000000000000000000000000F5
:100C000000000000000000000000000000000000E4
:100C100000000000000000000000000000000000D4
:100C200000000000000000000000000000000000C4
:100C30000000000041018B0A41018C0041018D0040
:100C400041018E0041018F0041019000410191005E
:100C5000410192004101930041019400410195003E
:100C6000410196004101970041019800410199001E
:100C70004103BF004103BE0020302A0000000000F5
:100C80000000000000000000000000000000000064
:100C90000000000000000000000000000000000054
:100CA0000000000000000000000000603002C700EB
:100CB0000000000000000000000000000000000034
:100CC0000000000000000000000000000000000024
:100CD0000000000000000000000000000000000113
:100CE00028000129704102C600C12AC128C12BC1B8
:100CF0002DC12EC12CC1294103710041036F004158
:100D0000036D0041036E004103700041036800C1A0
:100D1000264203690000C12741036B0041036C00B8
:100D2000C137C136C134C133C135C132410383003B
:100D300041037B0041037C0041037D00C12FC13092
:100D4000C1B141037E0041037F00410380004103A4
:100D500081004103820000E709F608DFFA8046E7D8
:100D600009F208DFFA803E88828C83E709F0A3DF6E
:100D7000FA8032E309F608DFFA8078E309F208DF47
:100D8000FA807088828C83E309F0A3DFFA8064899B
:100D9000828A83E0A3F608DFFA805889828A83E09A
:100DA000A3F208DFFA804C80D280FA80C680D4801B
:100DB0006980F28033801080A680EA809A80A880C3
:100DC000DA80E280CA803389828A83ECFAE493A3D2
:100DD000C8C582C8CCC583CCF0A3C8C582C8CCC561
:100DE00083CCDFE9DEE7800D89828A83E493A3F672
:100DF00008DFF9ECFAA9F0EDFB2289828A83ECFA8C
:100E0000E0A3C8C582C8CCC583CCF0A3C8C582C83E
:100E1000CCC583CCDFEADEE880DB89828A83E49379
:100E2000A3F208DFF980CC88F0EF60010E4E60C3BA
:100E300088F0ED2402B4040050B9F582EB2402B42A
:100E4000040050AF2323458223900DA773BB0106F6
:100E500089828A83E0225002E722BBFE02E32289D4
:100E6000828A83E49322BB010CE58229F582E58323
:100E70003AF583E0225006E92582F8E622BBFE0619
:100E8000E92582F8E222E58229F582E5833AF583B5
:100E9000E49322BB010689828A83F0225002F72262
:100EA000BBFE01F322BC000BBE0029EF8DF084FFD6
:100EB000ADF022E4CCF875F008EF2FFFEE33FEEC36
:100EC00033FCEE9DEC984005FCEE9DFE0FD5F0E95D
:100ED000E4CEFD22EDF8F5F0EE8420D21CFEADF05C
:100EE00075F008EF2FFFED33FD4007985006D5F061
:100EF000F222C398FD0FD5F0EA22C2D5EC30E70903
:100F0000B2D5E4C39DFDE49CFCEE30E715B2D5E418
:100F1000C39FFFE49EFE120EA5C3E49DFDE49CFC6E
:100F20008003120EA530D507C3E49FFFE49EFE2286
:100F3000C5F0F8A3E028F0C5F0F8E582158270024C
:100F40001583E038F022A3F8E0C5F025F0F0E58243
:100F5000158270021583E0C838F0E822E88FF0A40B
:100F6000CC8BF0A42CFCE98EF0A42CFC8AF0EDA430
:100F70002CFCEA8EF0A4CDA8F08BF0A42DCC382563
:100F8000F0FDE98FF0A42CCD35F0FCEB8EF0A4FE43
:100F9000A9F0EB8FF0A4CFC5F02ECD39FEE43CFCD8
:100FA000EAA42DCE35F0FDE43CFC2275F0087582F4
:100FB00000EF2FFFEE33FECD33CDCC33CCC58233E3
:100FC000C5829BED9AEC99E58298400CF582EE9BE8
:100FD000FEED9AFDEC99FC0FD5F0D6E4CEFBE4CD06
:100FE000FAE4CCF9A88222B800C1B90059BA002DA0
:100FF000EC8BF084CFCECDFCE5F0CBF97818EF2F59
:10100000FFEE33FEED33FDEC33FCEB33FB10D70387
:10101000994004EB99FB0FD8E5E4F9FA227818EF30
:101020002FFFEE33FEED33FDEC33FCC933C910D78F
:10103000059BE99A4007EC9BFCE99AF90FD8E0E49C
:10104000C9FAE4CCFB2275F010EF2FFFEE33FEED72
:1010500033FDCC33CCC833C810D7079BEC9AE89942
:10106000400AED9BFDEC9AFCE899F80FD5F0DAE424
:10107000CDFBE4CCFAE4C8F922E8600FECC313FC22
:10108000ED13FDEE13FEEF13FFD8F122ECF0A3ED0C
:10109000F0A3EEF0A3EFF022A8828583F0D083D0F6
:1010A000821210AF1210AF1210AF1210AFE473E43F
:1010B00093A3C583C5F0C583C8C582C8F0A3C58303
:1010C000C5F0C583C8C582C8228A838982E473E5D6
:1010D0007C2582F582E57B3583F583B57B048582AB
:1010E0007C2210AF0685827CF57B2285827CF57B95
:1010F000D2AF22E57C2582F582E57B3583F583221C
:10110000E3F5F009E208B5F06BDFF58067E3F5F091
:1011100009E608B5F05EDFF5805A87F009E608B504
:10112000F052DFF6804E87F009E208B5F046DFF6B0
:10113000804288828C8387F009E0A3B5F036DFF621
:10114000803288828C8387F009E493A3B5F025DF91
:10115000F5802188828C83E3F5F009E0A3B5F014D3
:10116000DFF5801088828C83E3F5F009E493A3B562
:10117000F002DFF402122F808780E9809080D48013
:101180003E8015806E807E809D80B7808D80A3809C
:10119000518074803C02123B89828A83ECFAE4938A
:1011A000F5F0A3C8C582C8CCC583CCE493A3C8C559
:1011B00082C8CCC583CCB5F076DFE3DEE1807089F0
:1011C000828A83E493F5F0A3E208B5F062DFF4804D
:1011D0005E89828A83E0F5F0A3E608B5F051DFF579
:1011E000804D89828A83E0F5F0A3E208B5F040DF04
:1011F000F5803C89828A83E493F5F0A3E608B5F094
:101200002EDFF4802A8002805789828A83ECFAE4F8
:1012100093F5F0A3C8C582C8CCC583CCE0A3C8C5EC
:1012200082C8CCC583CCB5F006DFE4DEE280007F67
:10123000FFB5F0020F2240027F012289828A83ECEF
:10124000FAE0F5F0A3C8C582C8CCC583CCE0A3C83A
:10125000C582C8CCC583CCB5F0D5DFE5DEE380CF51
:1012600089828A83ECFAE0F5F0A3C8C582C8CCC5B0
:1012700083CCE493A3C8C582C8CCC583CCB5F0AFFA
:10128000DFE4DEE280A988F0EF60010E4E60ABED96
:101290002402B404005098F582EB2402B4040050F8
:1012A0008E232345822390117773EF4E6012EF60F7
:1012B000010EEDBB010B89828A83F0A3DFFCDEFA0D
:1012C0002289F05007F709DFFCA9F022BBFEFCF3EE
:1012D00009DFFCA9F02220140330152EE49001CA86
:1012E000F0900198F0900190F0A3F0A3F0A3F0A388
:1012F000F0A3F0A3F0A3F0900199F09001CDF0904D
:1013000001CFF090019CF00216A49001A6E0FB64CE
:101310001160030215873009030215879001F7E079
:10132000540F6407600BA3E0540F640360030215BD
:10133000879001CDE04420F09001CAE0FC600302F8
:1013400013C8900294E0FE5403FFBF032490019061
:10135000E004F0E0D3941E500302170AE4F0900179
:10136000CA04F09001CDE04408F09001CF7401F080
:1013700022EE30E11F90028CE06019900192E004AF
:10138000F0E0D39414500302170AE4F09001CA74F9
:10139000020215D3BF022390028CE0701D900194CD
:1013A000E004F0E0D39432500302170AE4F0900115
:1013B000CA7403F09001CF14F022E4900190F090F1
:1013C0000192F0900194F022EC6401705590019824
:1013D000E0FF700E900294E05403600302170A02CB
:1013E0001657EF6401600302170A900191E004F0C0
:1013F000E0D3940A500302170A740AF0900294E0B2
:1014000054036401600302170A9001CAF090019826
:10141000F09001CDE054F7F0E49001CFF09001910D
:10142000F0229001CAE0FFB40216900294E020E19D
:101430000302162690028CE0600302170A021626A9
:10144000EF6403600302170A900198E0FF701790A1
:101450000294E05403600302170A90028CE06003D8
:1014600002170A021657EF64016003021565900225
:1014700094E05403FF6402704390028CE0703D904E
:101480000199F0900195E004F0E0D3940A50030232
:10149000170AE4F09001CFF09001987402F09001E7
:1014A000AFE0FE64026006EE600302170A9001AF2F
:1014B000E06402900102F09001AF8046EF64017099
:1014C0004590028CE0703F900199F0900196E00405
:1014D000F0E0D3940A500302170AE4F09001CFF031
:1014E0009001987402F09001C4E0FF64046006EF7C
:1014F000600302170A9001C4E06404900103F090B5
:1015000001C4F0D2072290028CE0603E900294E089
:1015100054037036900199F0900197E004F0E0D305
:10152000940A500302170AE4F09001CFF09001985A
:101530007402F090019CE0FF64086006EF60030213
:10154000170AEF640890019CF022E4900195F0A343
:10155000F0A3F0900199E004F0E0D394325003023C
:10156000170A0216BA900198E06402600302170A93
:1015700090028CE0600302170A900294E05403602A
:101580000302170A0216DAEB645560030216E33011
:1015900009030216E39001F7E0540F6407600BA300
:1015A000E0540F640360030216E39001CAE0705F29
:1015B000900294E030E125124FE7BF011F900193A4
:1015C000E004F0E0D39414500302170AE4F0900111
:1015D000CA7404F09001CDE04402F022900294E03D
:1015E00030E124124FE7EF701E900194E004F0E028
:1015F000D39432500302170AE4F09001CA7405F044
:101600009001CF7402F022E4900193F0A3F02290B5
:1016100001CAE0B4041D900294E030E109124FE7E2
:10162000EF600302170AE49001CAF09001CDE05484
:10163000FDF0229001CAE06405600302170A9001E0
:1016400098E07019900294E030E10302170A124FFB
:10165000E7EF600302170A90019804F022900198C6
:10166000E064017060900294E020E13D124FE7EFEA
:1016700064017035900199F0900196E004F0E0D398
:10168000940A500302170A9001987402F0E4900142
:1016900096F09001CFF09001A8E0FF6004648070A4
:1016A00069EF64809001A8F022E4900196F0900127
:1016B00099E004F0E0D394324050E4F09001CAF095
:1016C0009001988040900198E06402703D900294EF
:1016D000E020E136124FE7EF70309001CAF0900140
:1016E00098F022E49001CAF0900198F0900190F0F7
:1016F000A3F0A3F0A3F0A3F0A3F0A3F0A3F0900154
:1017000099F09001CDF09001CFF022E4900350F0D9
:10171000A3F0A3F0A3F078547C037D017BFF7A73E0
:101720007950FE7F08120E2778547C037D017B01DF
:101730007A02798C7E007F08120E279001AAE09031
:101740000353F09001A6E0FF64116005EF6455704B
:101750002B9001CAE0FF64036005EF6405701D7EF5
:10176000003023047F0880027F027D007B017A0322
:1017700079541212AA900353E054FCF09001A9E0AE
:10178000601D7E003023047F0880027F027D007B85
:10179000017A0379541212AA900353E054FCF030FA
:1017A000116EC211E49001A9F09001B0E0FD24FF98
:1017B000FFE434FFFEEF7803CEC313CE13D8F990C5
:1017C000035CF0ED145407A3F090035CE02454F59F
:1017D00082E43403F583C083C082E0FF90035DE0C0
:1017E000FE7401A806088002C333D8FC4FD082D013
:1017F00083F07E007F047D007B017A0179BF1212A5
:10180000AA7E007F047D007B017A0179B01212AAC2
:101810002023030218F090028BE030E3030218A4A7
:101820002008030218A4E4900350F0900350E0FF56
:10183000C39408506F74542FF582E43403F583E0A9
:10184000900352F0E4900351F0900351E0FFC394F1
:10185000085049EF90736493FF900350E0FE24FF1B
:10186000F582E43401F583E0FD900352E05DFDEF85
:101870005D602174542EF582E43403F583C083C087
:1018800082E0FF900351E090736493F4FEEF5ED02A
:1018900082D083F0900351E004F080AD900350E0DB
:1018A00004F0808778537C027D017B017A037954B0
:1018B0007E007F08120E27E4900350F0900350E062
:1018C000FF2453F582E43402F583C083C082E0FE36
:1018D000740E2FF582E43402F583E0FFEE4FD082E0
:1018E000D083F0900350E004F0E0B408CF02199DDB
:1018F000900289E030E30302197B30087EE4900314
:1019000050F0900350E0FFC39402506F74542FF5D1
:1019100082E43403F583E0900352F0E4900351F045
:10192000900351E0FFC394085049EF90736493FF14
:10193000900350E0FE24FFF582E43401F583E0FDDE
:10194000900352E05DFDEF5D602174542EF582E45A
:101950003403F583C083C082E0FF900351E09073AD
:101960006493F4FEEF5ED082D083F0900351E004E4
:10197000F080AD900350E004F0808778537C027DC6
:10198000017B017A0379547E007F02120E277E00CC
:101990007F067D007B017A0279551212AA2023036B
:1019A000021A2A90028BE030E403021A3D1251B26F
:1019B000EFD39401501A785B7C027D017B017A029F
:1019C00079257E007F08120E27E4900266F0806D74
:1019D000900354E0FCA3E0FDA3E0FEA3E0FF90022F
:1019E00025E0F8A3E0F9A3E0FAA3E05FFFEA5EFEDA
:1019F000E95DFDE85CFC90025B12108C900358E0FE
:101A0000FCA3E0FDA3E0FEA3E0FF900229E0F8A321
:101A1000E0F9A3E0FAA3E05FFFEA5EFEE95DFDE81E
:101A20005CFC90025F12108C8013785B7C027D015D
:101A30007B017A0279257E007F08120E279001A68D
:101A4000E0B4111E900207E030E717D212785B7CF9
:101A5000027D017BFF7A7379327E007F08120E27A8
:101A60008002C21290021EE0FF900353E04F9002EA
:101A700063F09001CDE0FF9001ABE04FFF90019C3F
:101A8000E04FFF9001A8E04F900264F0024F30E475
:101A90009003ACF0302905C229024CBE202B030272
:101AA0001DF0C22B303603021DF020210C2025032F
:101AB000021B55301E03021B557E007F107D007BEC
:101AC000017A0279D71212AA90036DE0606B90033D
:101AD0006EE0FF6064B4310D7B017A0279D7900328
:101AE000887403802090036DE0FFC394304028EF9A
:101AF000D39439502290036EE0FF7B017A0279D7AC
:101B00009003887401F0122E8D90036DE0FF7B012D
:101B10007A0279D8021BC890036EE0FF7B017A023B
:101B200079D79003887401F0122E8D90036DE0FF39
:101B30007B017A0279D8021BEE90036EE06003020B
:101B40001DF090036DE0FF7003021DF07B017A022F
:101B500079D7021C0E201E03021C167E007F207DFA
:101B6000007B017A0279C71212AA90036DE070031C
:101B7000021BF590036EE0FF607BB4311C7B017AA1
:101B80000279CF9003887403F0122E8D90036DE0DC
:101B9000FF7B017A0279D0802F90036DE0FFC39420
:101BA00030402CEFD39439502690036EE0FF7B0138
:101BB0007A0279CF9003887401F0122E8D90036D14
:101BC000E0FF7B017A0279D0900388740280439011
:101BD000036EE0FF7B017A0279CF9003887401F0F5
:101BE000122E8D90036DE0FF7B017A0279D0900375
:101BF000887401801D90036EE06003021DF0900365
:101C00006DE0FF7003021DF07B017A0279CFE49052
:101C10000388F0022E8D9003AC7408F09003ACE0C2
:101C2000FFC39418502074C72FF582E43402F58363
:101C3000E4F074DF2FF582E43402F583E4F09003DE
:101C4000ACE004F080D690036DE07003021D249098
:101C5000036EE07003021D24C39420405C9003BE19
:101C6000E0FF90036EE0FED39F504EEE75F009A4A6
:101C70002415F9745335F0FA9003A974FFF0A3EA20
:101C8000F0A3E9F078D27C027D019003A9E0FBA3E8
:101C9000E0FAA3E0F97E007F05120E279003A9E089
:101CA000FBA3E0FAA3E02405F9E43AFA78E77C0222
:101CB0007D017E007F04120E2790036DE0FFC39428
:101CC000205003021DF09003BEE0FEEFD39E4003C0
:101CD000021DF090036DE075F009A42415F974530A
:101CE00035F0FA9003A974FFF0A3EAF0A3E9F078C5
:101CF000DA7C027D019003A9E0FBA3E0FAA3E0F9FE
:101D00007E007F05120E279003A9E0FBA3E0FAA353
:101D1000E02405F9E43AFA78EF7C027D017E007F49
:101D200004020E2790036EE06003021DF090036D25
:101D3000E07003021DF075F009A42415F974533501
:101D4000F0FA9003A974FFF0A3EAF0A3E9F0A374FA
:101D50000BF09003ACE0FFC3941050429003A9E055
:101D6000FBA3E0FAA3E0F9120E4DFEC4540FFD747C
:101D7000C72FF582E43402F583EDF0EEC454F0FE93
:101D800074CF2FF582E43402F583EEF09003AAE4D9
:101D900075F001120F309003ACE004F080B49003B2
:101DA000AC7420F09003ACE0FFC394245042900345
:101DB000A9E0FBA3E0FAA3E0F9120E4DFEC4540F14
:101DC000FD74C72FF582E43402F583EDF0EEC454C0
:101DD000F0FE74CF2FF582E43402F583EEF0900329
:101DE000AAE475F001120F309003ACE004F080B467
:101DF00022E49003BCF09001AAE05403FFBF032E3D
:101E000090019AE060289001CBE004F0E0B41E233A
:101E1000E490019AF09001A97403F09001C6740156
:101E2000F0E49001CBF09001C8F0A3F08005E490BD
:101E300001CBF09001C6E070030221129001A9E0ED
:101E4000640360030221129001C9E004F07006905F
:101E500001C8E004F09001C8E0FEA3E0FFD3943293
:101E6000EE94004003021F647C007D03120EA5ED7A
:101E70004C700690019BE0F4F012367C78AC7C014B
:101E80007D017E007F02120E279001ACE0FF7016EC
:101E90009001C7E060109001CEEFF09001B57401A1
:101EA000F0E49001C7F09001B5E0603D9001CEE014
:101EB000FF9001ACE0FE6F60309001CEEEF090013B
:101EC000C5E004F0E0FF30E0209001ADE0FBEF243E
:101ED000FFFFE434FFFE7C007D02120EFA74BF2F78
:101EE000F58274013EF583EBF09001C5E064086073
:101EF000030221129001BFE09003BCF075F004A42E
:101F000024FCF582E5F034FFF583E0FF640160080E
:101F1000EF640360030221129003BCE075F004A497
:101F200024FDF974FF35F0FA7B0178C07C017D0156
:101F30007E007F03121286EF701ED2109001C8F04F
:101F4000A37432F090019A7401F09001C7F0E4900C
:101F500001B5F09001C5F0229001C8E4F0A37464CB
:101F6000F00220E29001C8E0FEA3E0FFC39464EE1B
:101F7000940040030220792010030220797C007D28
:101F800003120EA5ED4C700690019BE0F4F01236A2
:101F90007C78AC7C017D017E007F02120E279001CF
:101FA000ACE0FF70169001C7E060109001CEEFF03A
:101FB0009001B57401F0E49001C7F09001B5E060C4
:101FC0003C9001CEE0FF9001ACE0FE6F602F9001ED
:101FD000CEEEF09001C5E004F0E0FF30E01F90018C
:101FE000ADE0FBEF2401FFE433FE7C007D02120E26
:101FF000FA74BF2FF58274013EF583EBF09001C5B2
:10200000E0640660030221129003BDF09001BFE07E
:102010009003BDF0E0FF75F004A424FCF582E5F028
:1020200034FFF5837403F09001C0E0FE75F004EF17
:10203000A424FDF582E5F034FFF583EEF09001C1B4
:10204000E0FF9003BDE0FE75F004A424FEF582E5F8
:10205000F034FFF583EFF09001C2E0FF75F004EE7D
:10206000A424FFF582E5F034FFF583EFF0D20F9062
:1020700001C8E4F0A37467F0223010579001C5E066
:1020800070519001BFE09003BCF075F004A424FCF3
:10209000F582E5F034FFF583E09003BCB40114E071
:1020A00075F004A424FCF582E5F034FFF583740395
:1020B000F08012E075F004A424FCF582E5F034FF12
:1020C000F5837401F0D2049001C8E4F0A37467F0C2
:1020D000C21022C39001C9E094679001C8E0940047
:1020E00050079001CF7403F02290019A7401F09090
:1020F00001C7F0E49001C6F090019BF09001C8F098
:10210000A3F09001B5F09001C5F09001CFF09001DF
:10211000A9F022E49003BAF090019AE060641236CC
:102120007C78AC7C017D017E007F02120E2790013D
:10213000ACE06045A3E09003BAF075F004A424FC81
:10214000F582E5F034FFF583E06003B4FF239001EE
:10215000CBE004F0E0B40A2AE490019AF09001C6C2
:1021600004F0E49001CBF09003BAE09001BFF0805E
:10217000119001CF7403F08009E49001CBF090013D
:10218000CFF09001C6E070030222FC9001C9E00488
:10219000F070069001C8E004F09001C8E0FEA3E0F2
:1021A000FFD39432EE9400400302224A7C007D0368
:1021B000120EA5ED4C700690019BE0F4F012367CF7
:1021C00078AC7C017D017E007F02120E279001AC6D
:1021D000E0FF70169001C7E060109001CEEFF09024
:1021E00001B57401F0E49001C7F09001B5E0603CE6
:1021F0009001CEE0FF9001ACE0FE6F602F9001CE29
:10220000EEF09001C5E004F0E0FF30E01F9001AD7A
:10221000E0FBEF2401FFE433FE7C007D02120EFAA6
:1022200074BF2FF58274013EF583EBF09001C5E099
:10223000640560030222FC9001C704F0E49001B53C
:10224000F09001C8F0A37432F022D39001C9E09459
:10225000359001C8E09400500F9001C5E06405601E
:10226000079001CF7403F0229001C5E06405706708
:102270009003BBF0D20F9001BFE09003BBF0E0FFF2
:1022800075F004A424FCF582E5F034FFF5837403B3
:10229000F09001C0E0FE75F004EFA424FDF582E5A6
:1022A000F034FFF583EEF09001C1E0FF9003BBE056
:1022B000FE75F004A424FEF582E5F034FFF583EF0B
:1022C000F09001C2E0FF75F004EEA424FFF582E572
:1022D000F034FFF583EFF0E49001CFF090019A0421
:1022E000F09001C7F0E49001C6F090019BF09001DE
:1022F000C8F0A3F09001B5F09001C5F022E490037E
:10230000CAF012367C78AC7C017D017E007F02121F
:102310000E279001ACE0FB607990019AE060739029
:1023200001ADE09003CAF075F004A424FCF582E549
:10233000F034FFF583E0640370589001A97404F051
:102340009001C67401F0E490019AF09003CAE09005
:1023500001B0F075F004A424FDF582E5F034FFF53A
:1023600083E09001B1F09003CAE0FF75F004A4246B
:10237000FEF582E5F034FFF583E09001B2F075F0F0
:1023800004EFA424FFF582E5F034FFF583E090012B
:10239000B3F09001C6E070030224CB9001C9E004C1
:1023A000F070069001C8E004F09001C8E0FEA3E0E0
:1023B000FFD3941EEE940040030224657C007D034D
:1023C000120EA5ED4C700690019BE0F4F0EB701935
:1023D0009001C7E060139001ACE09001CEF0900155
:1023E000B57401F0E49001C7F09001B5E07003020C
:1023F00024D09001CEE0FF9001ACE0FE6F700302AC
:1024000024D09001CEEEF09001C5E004F0E0FF3062
:10241000E01F9001ADE0FBEF2401FFE433FE7C0000
:102420007D02120EFA74BF2FF58274013EF583EB24
:10243000F09001C5E0640660030224D078B17C010D
:102440007D017B017A0179C0FE7F03121286EF7055
:102450000A9001C3E07004D21104F09001C8E4F0C6
:10246000A3741EF022D39001C9E094219001C8E02A
:102470009400500D9001C3E070079001CF7403F0F9
:102480002290019A7401F09001C7F0E49001C6F027
:1024900090019BF09001C8F0A3F09001B5F090017D
:1024A000C5F09001CFF09001C3F0201123FE7F040E
:1024B000FD7B017A0179BF1212AA7E007F047D00A4
:1024C0007B017A0179B01212AA8000E49001A9F090
:1024D00022900392EBF0A3EAF0A3E9F0E4FFA3F06B
:1024E000A3F0A3F0FD303306C2339002C6F02021E2
:1024F00006202503022588E4FF74C92FF582E43401
:1025000002F583E0FE74C72FF582E43402F583EE12
:10251000F00F74C92FF582E43402F583E0FE74C72E
:102520002FF582E43402F583EEF00FEFC3941E40E2
:10253000C89002C6E0C39410400302267D90039227
:10254000E0FBA3E0FAA3E0F99002C6E0FE75F0021A
:10255000A4F58285F083120E669002E5F090039256
:10256000A3A375F002EEA42401F582E435F0F5830F
:10257000120E669002E6F09002C6E004F0E06410ED
:10258000600302267D02267A9002C6E0FEC3941004
:10259000400302267DEEFB7A007E007803CEC31353
:1025A000CE13D8F9900396F0EB5407A3F0E4FF7430
:1025B000CF2FF582E43402F583E05480C413131363
:1025C0005401FD74C72FF582E43402F583E025E061
:1025D0004DFE74C72FF582E43402F583EEF074D714
:1025E0002FF582E43402F583E05480C413131354AE
:1025F00001FD74CF2FF582E43402F583E025E04D30
:10260000FE74CF2FF582E43402F583EEF09003924E
:10261000E0FBA3E0FAA3E0F9900396E0F58275836E
:1026200000120E66FE900397E0FDEEA805088002FA
:10263000C333D8FC5480C41313135401FD74D72F33
:10264000F582E43402F583E025E04DFE74D72FF5E2
:1026500082E43402F583EEF0900396E02402F0EF7A
:10266000B407027F170FEFC3942050030225AF90E9
:1026700002C6E004F0E0B41004E4F0D2352278A100
:102680007C037D017BFF7A7379587E007F02120EF6
:102690002778A37C037D017BFF7A73795A7E007FC4
:1026A00002120E27300D6A78A17C037D017B017A2E
:1026B0000179007E007F02120E27900104E0FEA344
:1026C000E0FF7B017A0079007D047C011234B6EFD3
:1026D00060E8900105E02400FF900104E03401FE71
:1026E0007B017A0379A37D027C001239EAEF700343
:1026F00002282978A17C037D017B017A0379A37EDE
:10270000007F02121286EF6003022829D20CC20D4C
:1027100022303F6878A17C037D017B017A01790238
:102720007E007F02120E27900104E0FEA3E0FF7BF3
:10273000017A0079007D047C011234B6EF60E890E4
:102740000105E02402FF900104E03401FE7B017AE0
:102750000379A37D027C001239EAEF700302282975
:1027600078A17C037D017B017A0379A37E007F023F
:10277000121286EF6003022829C23F2230076278D6
:10278000A17C037D017B017A0179027E007F021228
:102790000E27900104E0FEA3E0FF7B017A007900A0
:1027A0007D047C011234B6EF60E8900105E024025C
:1027B000FF900104E03401FE7B017A0379A37D02DE
:1027C0007C001239EAEF606178A17C037D017B0116
:1027D0007A0379A37E007F02121286EF704BC20744
:1027E00022201D1E300F1B900104E0FEA3E0FF7BA2
:1027F000017A0079007D047C011234B6EF60E8C2F2
:102800000F22900264E020E72020E31D30041A909C
:102810000104E0FEA3E0FF7B017A0079007D047CE7
:10282000011234B6EF60E8C20422E4789BF630135C
:102830002E900378E0B40118A3E024FE600C04603D
:102840000302298B12479902298B1247FC02298B1C
:10285000900378E0600302298B1249D502298B90FE
:10286000026BE0FF640970467B017A02793CEF1449
:10287000FD12514890026BE0243BF582E43402F5EE
:1028800083E06F7029789BF6789BE6FF243CF58205
:10289000E43402F583E0F4FE74252FF582E434027B
:1028A000F583EEF006E6B408DF900374804D9003E4
:1028B00078E06403704A90026BE0FD641770417B1E
:1028C000017A02793C124D08EF4E7034789BF6780D
:1028D0009BE6FF243FF582E43402F583E0F4FE74C6
:1028E000252FF582E43402F583EEF006E6B410DF1E
:1028F00090024FE0900235F0900375E004F0801EE6
:10290000900378E0702790026BE0FDB4171F7B0105
:102910007A02793C124D08EF4E70121249D5C21A54
:10292000E490037AF0C21C900373F0800F9003735D
:10293000E004F0E4900375F0900374F0900374E009
:10294000C394644024A3E0FF700AD2139003790477
:10295000F0E4802BEFC3945A4029D213900379748A
:1029600002F0E4900375F08016900375E0C3946460
:102970004011D2139003797402F0E4900375F09043
:102980000374F0301305E4900378F0E490026CF0E7
:10299000C23D2290FFFB1210CF857B83857C82E4B1
:1029A000F0A3F0857B83857C82A3A3F090000312C3
:1029B00010F3E4F09000041210F3E4F0857B8385BB
:1029C0007C82F0857B83857C82E0FFC39405400395
:1029D000022A58EF25E0240AF808E61618700116B6
:1029E0001486064E7066857B83857C82E0FF25E039
:1029F000246FF582E43471F583E493FC740193FD54
:102A0000EF25E0240AF8A60408A605857B83857CCB
:102A100082E090717F93857B83857C82A3F0857BA8
:102A200083857C82A3E0FF551A6005EF4208801C75
:102A3000857B83857C82A3E0FF551B6005EF4209FF
:102A4000800A857B83857C82A3E0421B857B83850E
:102A50007C82E004F00229C31254318067900003A5
:102A60001210F3E0FF857B83857C82A3A3E0FEC385
:102A70009F5075EE14FF9000041210F3EFF0125403
:102A8000319000041210F3E090717F93FFF4521B19
:102A9000EF421A12542E9000041210F3E075F00366
:102AA000A42413F582E43403F583A3E0FAA3E0F948
:102AB0001210C91254319000041210F3E090717F8B
:102AC00093F4521AE51B90718793857B83857C82F2
:102AD000A3A3F0E51A90718793FF9000031210F3FF
:102AE000EFF012542E022A5D9000050210CFE49000
:102AF00003C3F0301354900378E014603714604639
:102B000024027044900379E0FFB401129001D17463
:102B100020F0A374D9F0A3744DF0C2188071EFB403
:102B200002109001D17421F0A374D8F0A3744CF07A
:102B3000D218805B9001D17427F0A374DEF0A374E7
:102B40004AF0C2188049804F8061900378E0146099
:102B50001C14602B146040240370509001D1742029
:102B6000F0A374D9F0A3744DF0C21880229001D163
:102B70007427F0A374DEF0A3744AF0C2188010909A
:102B800001D17421F0A374D8F0A3744CF0D2189042
:102B90000378E004F080199001D17422F0A374DB73
:102BA000F0A3744FF0D218D21B8000E4900378F0A9
:102BB0002018419001F8E09001D4F09001FAE090E3
:102BC00001D5F09001F9E09001D6F078D77C017D35
:102BD000017B017A0179FF7E007F05120E279002AA
:102BE00007E09001DCF09001DE740DF0E47899F6D6
:102BF00008F68028E49001D4F0A3F0301B10C21B2B
:102C0000A3F0A3F0A3F09001DE740AF08006900117
:102C1000DE7407F0789676FF789876FF120050E41D
:102C20009001DFF0301F0443AA02229003C3E5ACF9
:102C3000F075AC01D299E0F5AC22E4FD90037CE0A4
:102C4000FC04F0EC64026003022D71F090036FE06D
:102C5000FC20E403022CE1303603022D7120210315
:102C600030252D9002C7E0FEA3E0FDE4FF74C92FDC
:102C7000F582E43402F583E0FB74C72FF582E43477
:102C800002F583EBF00FEFB40CE39002D3022D1E9C
:102C90009002C7E0FEE4FF74C82FF582E43402F529
:102CA00083E0FB74C72FF582E43402F583EBF00F69
:102CB000EFB407E39002DFE09002CEF07F1874C813
:102CC0002FF582E43402F583E0FB74C72FF582E42C
:102CD0003402F583EBF00FEFB41FE39002E6EEF061
:102CE00022EC20E503022D71303603022D712021E4
:102CF000033025309002D3E0FEA3E0FD7F0D74C5C4
:102D00002FF582E43402F583E0FC74C72FF582E4EA
:102D10003402F583ECF01FEFB401E39002C7EEF04C
:102D2000A3EDF0229002E6E0FE7F1F74C62FF5822D
:102D3000E43402F583E0FD74C72FF582E43402F534
:102D400083EDF01FEFB418E39002CEE09002DFF0C5
:102D50007F0774C62FF582E43402F583E0FD74C763
:102D60002FF582E43402F583EDF0DFE69002C7EE42
:102D7000F022E49003C5F0FE900207E0541CFF909F
:102D800001CFE04F9003C5F06404701C302307901E
:102D9000028BE020E30A30210A900289E030E3034D
:102DA000022E70E4FE022E8A9003C5E0FFB40303F6
:102DB000022E759001A6E0641160099001CAE070CE
:102DC00003022E8A9003C5E0FF24FE602F24FA60E0
:102DD0003D24FC604C24FC605B24FC606B24FC60A4
:102DE0007C24FC7003022E70241B6003022E88904A
:102DF000039B7405F0E4A3F07B0580359003C5E0E8
:102E0000FFE490039BF0A37404F0E4FB80239003A1
:102E1000C5E0FF90039B7405F0E4A3F0FB7D058003
:102E2000609003C5E0FF90039B740FF0E4A3F07B78
:102E30000AFD804D9003C5E0FF90039B7402F0A350
:102E400014F07B057D0380399003C5E0FF90039B60
:102E5000740CF0A37401F07B057D0380249003C5FE
:102E6000E0FF90039B7402F0A3F07B057D038011CB
:102E70009003C5E0FFE490039BF0A37403F0E4FB30
:102E8000FD122FA6AE078002E4FEAF062290038556
:102E9000EBF0A3EAF0A3E9F0EFC394205003022F74
:102EA000A59003BEE0FDEFD39D4003022FA5EF7573
:102EB000F008A42475F9745535F0FA90038974FF6D
:102EC000F0A3EAF0A3E9F0E4FE900388E0FF705578
:102ED000A3E0FBA3E0FAA3E0F98E82758300120E53
:102EE0006654F0C4540FFD900385E0FBA3E0FAA301
:102EF000E0F9ED120E93900389E0FBA3E0FAA3E062
:102F0000F98E82758300120E66540FC454F0FD9042
:102F10000385E0FBA3E475F001120F30A9F0FAED90
:102F2000120E93806DEF5403FFBF0224900389E0DB
:102F3000FBA3E0FAA3E0F98E82758300120E6625EA
:102F4000E0FD900385E0FBA3E0FAA3E0F9ED803516
:102F5000900389E0FBBF0312A3E0FAA3E0F98E829D
:102F6000758300120E66C313800EA3E0FAA3E0F986
:102F70008E82758300120E66FF900385E0FBA3E04E
:102F8000FAA3E0F9EF120E93900386E475F00112B4
:102F90000F30900386E475F001120F300EEE6408D6
:102FA0006003022EC92290039CE0FEB4030D900141
:102FB0000AEFF0C200C201C2028078EEB4040E90A3
:102FC000010AEFF0C200C201C20202307290010A8F
:102FD000E06F600FEFF0200308C200C201C2028060
:102FE00002C20320005590010AEFF0D20090039C2A
:102FF000E07017EDAE036001FE900109EEF0ED7E8A
:103000000860027E0C900108EEF090039CE0FEB494
:103010000114900109EDF0EF900108B41405741C3F
:10302000F08003740CF0EE640260030230B490018F
:1030300009EBF09001087408F0807920013C9001C0
:1030400009E014F0706ED20190039CE0603FB4017F
:1030500014900109EBF0EF900108B414057418F016
:1030600080037408F090039CE064027047900109AB
:10307000EDF0900108740CF0803A20021F900109D5
:10308000E014F0702FD20290039CE0601F90039B2D
:10309000E0900109F0E4900108F08018900109E047
:1030A00014F0E024FFFFE434FF4F7008D203C200A5
:1030B000C201C202900108E0FF22E49003CBF0209D
:1030C0002A030231A8D22790036BE0B40700400323
:1030D0000231A29030DAF82828730230EF02310270
:1030E00002312102314002315C023179023190908B
:1030F000036FE054CFF0D228D22DE4900371F00298
:10310000318990036CE0FF04F0EF649160030231B9
:10311000C4C22DF01252D390036BE004F0E4FD80A2
:103120001C90036CE0FF04F0EF641E60030231C4E6
:10313000F01252D390036BE004F07D01E4FF80367F
:1031400090036CE0FF04F0EF641E7078F01252D32D
:1031500090036BE004F0E4FD7F01801A90036CE0C3
:10316000FF04F0EF641E705CF01252D390036BE02A
:1031700004F07D017F010241BB90036CE0FF04F08D
:10318000EF641E703FF01252B490036BE004F02223
:1031900090036CE0FF04F0EF641E7028F01252D32D
:1031A0008000E490036BF02290036BE0600BE4F08E
:1031B000A3F0C2271252D38005302708C227D22895
:1031C000D22BC22D22900371E0540FFF90036FE0C9
:1031D000FE54306014EE20E610EF64026009EF64E4
:1031E000036004EFB40902E4FF90027EE04F900315
:1031F00083F0540F907374937009201506202D03EB
:103200000232B6D236202F0302329230317330357B
:103210005090037EE0543FFF900380E0FD1246C9CA
:1032200090037FEFF0A3E004F0EFF47032E014F0CD
:1032300090037F74BBF0900381E004F0E0FFB402E0
:1032400003302407EFB40313302410E4900381F01B
:10325000C22FC236D23012524F8006C2358002C20F
:103260003590037DE004F0B40117E4F090037FE0B3
:1032700075F020A42455F9745035F0FA7BFF122420
:10328000D190037EE0FF900383E06F543F6039C22A
:103290002F22D22FD233D235900383E090037EF0D9
:1032A000E4900380F0A3F0A3F0FE7F30FD7B017A71
:1032B0000279C70212AA303606C236C22F80033006
:1032C0003006C230D22BD2282290032B12108C90C1
:1032D000032FE0FF12539190026D302209121098D3
:1032E00001312D008007121098016E36009001D038
:1032F0003023057401F080037402F09001D0E0FFE8
:10330000E4FCFDFE90026DE0F8A3E0F9A3E0FAA36F
:10331000E0FB120F5CC004C005C006C007E47F20BC
:10332000FEFDFC90032BE0F8A3E0F9A3E0FAA3E094
:10333000FB120F5CA804A905AA06AB07D007D006AC
:10334000D005D004120FE7C3E49FFFE49EFE740192
:103350009DFDE49CFC78081210798FCB9001D0E0A1
:10336000FFE4FCFDFE90026DE0F8A3E0F9A3E0FAB3
:10337000A3E0FB120F5CC004C005C006C007E47FD9
:1033800020FEFDFC90032BE0F8A3E0F9A3E0FAA3F4
:10339000E0FB120F5CA804A905AA06AB07D007D072
:1033A00006D005D004120FE7C3E49FFFE49EFE742D
:1033B000019DFDE49CFCE48FCA75C83443B81043FA
:1033C000B71043A810020056EF14600C146061247B
:1033D0000260030234B58056900208E0605090030A
:1033E00079E064027042300E1EC20E785B7C027D72
:1033F000017B017A027925FE7F08120E27900235A3
:10340000E025E054FE801DD20E785B7C027D017BBE
:10341000017A02792D7E007F08120E27900235E096
:1034200025E04401FF02485F900379E080748072D8
:10343000900208E0606C900379E064027042300E04
:103440001EC20E785B7C027D017B017A027925FE2B
:103450007F08120E27900235E025E054FE801DD231
:103460000E785B7C027D017B017A02792D7E007FE4
:1034700008120E27900235E025E04401FF02000EFD
:10348000900379E0785B7C027D017B017A027925EB
:103490007E007F08B40109120E27E4900266F02234
:1034A0008010785B7C027D017B017A0279257E00A9
:1034B0007F08120E272290035EEEF0A3EFF0A3EC3C
:1034C000F0A3EDF0A3EBF0A3EAF0A3E9F0E4A3F09E
:1034D000A3F0A3F0900360E0FEA3E0FF90035EE0A2
:1034E000FCA3E0FD2FFFEC3EFEA3E0FAA3E0FBD33C
:1034F0009400EA9402501FEB4A601B900104E0FA2A
:10350000A3E0FBC3ED9BEC9A400C900107E09F9079
:103510000106E09E5002807690035EE0FEA3E0FF8D
:10352000124D99EF6401706690036504F0E4A3F016
:10353000A3F0900360E0FEA3E0FFC3900367E09F69
:10354000900366E09E504C90035EE0FEA3E0FF9087
:103550000362E0FBA3E0FAA3E0F9120E4DFD12486E
:10356000C0EF7002802990035FE004F070069003C2
:103570005EE004F0900363E475F001120F309003F5
:1035800067E004F070AC900366E004F080A4E4907F
:103590000365F0900365E0FF22E49003A5F0303668
:1035A0000302367B2021033025407E007F107D0002
:1035B0007B017A0279C71212AA90036FE030E410FF
:1035C0007B017A0279C7E4900388F07F5D122E8D2B
:1035D00090036FE020E50302367B7B017A0279C716
:1035E000E4900388F07F5E022E8DE49003A5F090B6
:1035F00003A5E0FFC39408502074C72FF582E4347C
:1036000002F583E4F074DF2FF582E43402F583E4FD
:10361000F09003A5E004F080D690036FE0FF30E463
:103620000E9003A674FFF0A37456F0A3745AF0EF43
:1036300030E50E9003A674FFF0A37456F0A37463F4
:10364000F0EF5430603578CA7C027D019003A6E02B
:10365000FBA3E0FAA3E0F97E007F05120E2790039A
:10366000A6E0FBA3E0FAA3E02405F9E43AFA78DF48
:103670007C027D017E007F04120E2722E49003402D
:10368000F0A3F0A3F0A3F0A3F0A3F078487C037DAF
:10369000017BFF7A73795CFE7F08120E2790028C03
:1036A000E0FCA3E0FDA3E0FEA3E0FF9003481210BE
:1036B0008C900290E0FCA3E0FDA3E0FEA3E0FF906D
:1036C000034C12108C9003453023057408F08003DE
:1036D0007402F0E4900340F0900345E0FF90034053
:1036E000E0FEC39F504F74482EF582E43403F58307
:1036F000E0900342F0E4900341F0900341E0FFC307
:1037000094085029A3E0FE30E014A3E004F0EF0495
:10371000FF900340E075F008A42F900344F0EEC33F
:1037200013900342F0900341E004F080CD900340F9
:10373000E004F080A3900343E0B4010F90034674CB
:1037400001F0900344E09003478006E4900346F0C4
:10375000A3F07B017A03794622E4FF201D0302389F
:10376000149001F8E0540F640160030237F29001F5
:10377000A904F0A3E05403FEBE03189001B4E004D2
:10378000F0E064326003023834F09001CF7403F04B
:10379000D20A22300A59E4FF75F004EFA42400F5A0
:1037A00082E5F03400F5837403F0EF04FE75F00455
:1037B000EFA42401F582E5F03400F583EEF075F016
:1037C00004EFA42402F582E5F03400F583EEF075F1
:1037D000F004EFA42403F582E5F03400F583EEF065
:1037E0000FEFB440B3D20FC20AE49001CFF022022F
:1037F00021139001F7E0540F64076008A3E0540F11
:10380000FFBF03099001A97402F0023E819001A953
:103810007405F0229001F7E0540F6407600BA3E0F9
:10382000540F64036003121DF19001A9E06403606A
:10383000031222FD22C0E0C0F0C083C082C0D07558
:10384000D000C000C001C002C003C004C005C00653
:10385000C007900336E4F0301F4DE5AA30E02B534B
:10386000AAFE1253B9303D030238F590026CE0C352
:10387000941740030238F5E0FF04F0743C2FF58202
:10388000E43402F583E59AF0806BE5AA30E16653F3
:10389000AAFD9001DEE0FFA3E0C39F50051253DDB7
:1038A0008053120018804E900336E5ACF075AC01E1
:1038B000309824C2981253B9203D3490026CE0C372
:1038C0009417502BE0FF04F0743C2FF582E434028F
:1038D000F583E599F08018309915C2999001DEE0E2
:1038E000FFA3E0C39F50051253DD80031200189020
:1038F0000336E0F5ACD007D006D005D004D003D015
:1039000002D001D000D0D0D082D083D0F0D0E0322D
:10391000300B030239E9302368E4FE75F004EEA4AD
:103920002400F582E5F03400F583E0FF64016004D3
:10393000EFB40321EE131313541F24B6F582E434BD
:1039400001F583C083C082E0FDEE5407907340937D
:10395000FCED4C8020EE131313541F24B6F582E4C3
:103960003401F583C083C082E0FDEE5407907340BC
:1039700093F4FCED5CD082D083F00EEEB4409C80DA
:1039800066E4FE75F004EEA42400F582E5F0340050
:10399000F583E0FF64016004EFB40321EE13131319
:1039A000541F24B6F582E43401F583C083C082E05D
:1039B000FDEE540790734093FCED4C8020EE131302
:1039C00013541F24B6F582E43401F583C083C0820A
:1039D000E0FDEE540790734093F4FCED5CD082D090
:1039E00083F00EEEB4109CD20B2290032BEEF0A3CA
:1039F000EFF0A3ECF0A3EDF0A3EBF0A3EAF0A3E962
:103A0000F0E4A3F0A3F0A3F090032DE0FEA3E0FF09
:103A100090032BE0FCA3E0FD2FFFEC3EFEA3E0FAB9
:103A2000A3E0FBD39400EA9402501FEB4A601B9082
:103A30000104E0FAA3E0FBC3ED9BEC9A400C90017B
:103A400007E09F900106E09E5007E4900332F0806B
:103A500064E4900333F0A3F090032DE0FEA3E0FFB5
:103A6000C3900334E09F900333E09E504290032BB9
:103A7000E0FEA3E0FF124F6E90032FE0FBA3E0FAFD
:103A8000A3E0F9EF120E93900330E475F001120FEA
:103A90003090032CE004F0700690032BE004F090CB
:103AA0000334E004F070B1900333E004F080A99097
:103AB00003327401F0900332E0FF229003B5E0146A
:103AC0006031147003023B4A24026003023B89E523
:103AD00074B413058576998017E574C39413500860
:103AE000747D2574F8E66276747D2574F8E6F599A0
:103AF000057422E574C39414503BE574B4130A852D
:103B00007699E57A6576FF801AE574C394135008B8
:103B1000747D2574F8E66276747D2574F8E6F5996F
:103B2000657AFFEF906F6F936578F57AEF90706F1D
:103B300093F5788012E574B41405857A998008E5C8
:103B400074B41503857899057422E57324FEFEE5A7
:103B500074C39E501C747D2574F8E6FD657AFF9051
:103B60006F6F936578F57AEF90706F93F578ED80CD
:103B700010EEB57404E57A8008E57314B57408E5B1
:103B800078A2D0929BF5990574229001A9E0B40225
:103B90001812391078FF7C017D017B017A0179B61A
:103BA0007E007F08120E278002C20B9001C6E060E3
:103BB0001390019BE09002076006E04401F080044E
:103BC000E054FEF0789D7C017D017B017A0179FF54
:103BD0007E003023547F04120E2778A27C017D01E1
:103BE0007B017A0279037E007F04120E27122D7268
:103BF000900207E054034F9001A1F0E0FEC00612CE
:103C00005379D0E04F9001A1F0E0FEC00612456E5E
:103C1000D0E04FFF9001A1F0900208E05480FEC375
:103C2000134F9001A1F00250D57F02120E27122DE2
:103C300072900207E054034F90019FF0E0FEC0062F
:103C4000125209D0E04F90019FF0124BDE227D010D
:103C50007B007E00120E27E490033BF0302312908D
:103C6000028BE030E40B2012089003B5E0FF123322
:103C7000C89003B5E014601F146034240270757896
:103C80007D7C007D007B017A0279537E007F1312D8
:103C90000E27757314805D787D7C007D007B017A32
:103CA0000279537E007F13120E277573168045909C
:103CB00001CCE0787DF6087665900208E030E61EDB
:103CC000900379E0B40217087C007D007B017A0242
:103CD00079537E007F14120E277573188016787F33
:103CE0007C007D007B017A0279537E007F13120EE7
:103CF00027757317E4F5767578FF757AFFF57412FA
:103D0000540090033BE5ACF0E4F5ACD299E0F5AC9F
:103D1000229003B5E014601914603024026003029D
:103D20003DA2E57164146003302277E575707380FD
:103D300015E57164166003302268E5757064E577F7
:103D40007060E579705C12465A8057E571641770AF
:103D500051E577704DE5797049302223E55AB4DC9E
:103D60001EE55BB46519D23CD21978E07C017D0177
:103D70007B007A00795C7E007F13120E278023205F
:103D8000230330211D9001CCE0B55A16E55BB465E4
:103D900011D23CD21978F77C017A00795C7F13123A
:103DA0003C4EC214E4900376F0301906C215A3F01D
:103DB0008006900377E004F0E4F572C23EF5757575
:103DC00077FF7579FF9003B5E0900372F022EF540E
:103DD00007B408004003023E6D903DE0F8282873C8
:103DE000023DF8023DFA023E07023E14023E29025D
:103DF0003E36023E4B023E5880739001A67422F07C
:103E00009001CC74DE80719001A67433F09001CCE7
:103E100074DF800B9001A67444F09001CC74E0F044
:103E2000D2089001AE7401F0229001A67455F09072
:103E300001CC74E1800B9001A67466F09001CC7403
:103E4000E2F0C2089001AE7402F0229001A67477ED
:103E5000F09001CC74E3800B9001A67488F090017F
:103E6000CC74E4F0D2089001AE7403F0229001A665
:103E70007411F09001CC74DDF0C208E49001AEF052
:103E800022E49003C9F012367C78AC7C017D017E7F
:103E9000007F02120E279001ACE0607DA3E090034A
:103EA000C9F075F004A424FCF582E5F034FFF58335
:103EB000E0FF64016005EF640370559001C6740172
:103EC000F09001CBE004F0E0FF75F00384E5F070C2
:103ED0000CEFC39432500690019BE0F4F09001CBBC
:103EE000E0643270459001C6F090019BF09001CBE8
:103EF000F09001CF7403F09003C9E075F004A4249E
:103F0000FCF582E5F034FFF583E4F0C20BD20F221A
:103F10009001CF7403F0E4800DE49001CFF09001A4
:103F2000CBF090019BF09001C6F022E52825E0241B
:103F30002AFF90033AEFF0E4F51CF51DF51EF51F7E
:103F400020250330213590033AE0F8E6F51DE8041A
:103F5000F8E6F51EE4F51C125023051CE51CC3947D
:103F60000840F4E4F51CE51C90736493551EFF12A1
:103F7000502C051CE51CC3940840EB3024569003DC
:103F80003AE0FFF8E6F51DE82408F8E6F51EEF2410
:103F900010F8E6F51FE4F51C125023051CE51CC3C0
:103FA000940840F4E4F51CE51C90736493551EFFDF
:103FB00012502C051CE51CC3940840EBE4F51CE5ED
:103FC0001C90736493551FFF12502C051CE51CC3F5
:103FD000940840EB2290032B12108C301F4875A6DA
:103FE0001490032FE0600575AAD0800375AA50E4F1
:103FF0007F20FEFDFC90032BE0F8A3E0F9A3E0FA9C
:10400000A3E0FB120F5CA804A905AA06AB07900366
:1040100030E0FCA3E0FDA3E0FEA3E0FF120FE7EF1A
:10402000F404F5BA804CE4F5AC759A1C75AC0190BB
:10403000032FE060054398D08003439850E47F103D
:10404000FEFDFC90032BE0F8A3E0F9A3E0FAA3E067
:10405000FB120F5CA804A905AA06AB07900330E089
:10406000FCA3E0FDA3E0FEA3E0FF120FE7EFF404E2
:10407000F59A43AD1043AF1043AE1002001878FF1D
:10408000E4F6D8FD9000007FFF7E04E4F0A3DFFC9F
:10409000DEFA757B04757C0075819C0240D90200B4
:1040A00003E493A3F8E493A34003F68001F208DF4E
:1040B000F48029E493A3F85407240CC8C333C454F0
:1040C0000F4420C8834004F456800146F6DFE480A4
:1040D0000B01020408102040809007BBE47E01938E
:1040E00060BCA3FF543F30E509541FFEE493A36076
:1040F000010ECF54C025E060A840B8E493A3FAE4D1
:1041000093A3F8E493A3C8C582C8CAC583CAF0A321
:10411000C8C582C8CAC583CADFE9DEE780BEE4F944
:104120009003B8F0A3F0FD7C023023027C08E4FF8A
:10413000EFC39C5079748C2FF582E43402F583E050
:104140009003B9F0E4FEEE90736493FB9003B9E042
:104150005B6015ED25E0240BF582E43401F583E482
:1041600075F001120F308010ED25E0240BF582E48C
:104170003401F583E4F0A3F0ED25E0240BF582E4AF
:104180003401F583E0FAA3E0C39458EA94024015A1
:10419000ED25E0240BF582E43401F5837402F0A3ED
:1041A0007458F079800D0EEEB4089B0F8082E9B44C
:1041B0008004D2098002C209AF0122E4FCFB202165
:1041C00003302538EF7020ED7C027001FCAE04EE68
:1041D000C394205076742A2EF876FF742B2EF8762E
:1041E000FF74042EFE80E8ED7B5570027BAAE4FE8E
:1041F000742A2EF8A6030EEEB420F522EF7038EDE7
:104200007C017001FCAF04AE07EEC39408503C740F
:104210002A2EF876FF74322EF876FF743A2EF8764E
:10422000FF74422EF876FF744A2EF876FF74522EF1
:10423000F876FF0E0E80D2ED7B5570027BAAE4FE6D
:10424000742A2EF8A6030EEEB430F522E49003ADE6
:10425000F0A3F0A3F09003AEE580F0A3E5A0F0E4B6
:104260009003ADF09003ADE0FFC3940A5061EF44BA
:1042700018F5A01254099003ADE0F5A01254097589
:1042800080FF9003ADE0FFC39406400EE580F4FE8E
:10429000748A2FF582E4340280169003ADE0FFC3E8
:1042A0009404E5804010F4FE74902FF582E434020B
:1042B000F583EEF08011F4FF9003ADE0248CF582DD
:1042C000E43402F583EFF09003ADE004F0809590C4
:1042D00003AEE0F580A3E0F5A022E4FF900208E041
:1042E00030E052200C4B90018EE0A3F090018DE065
:1042F000FEA3F0900209E090018DF06E70679001CE
:104300008FE0FE90018EE06E705B900100E0FE9009
:10431000018DE0FD6E6016D20D900100EDF0A374EA
:1043200001F0E490018DF0A3F0A3F080387F30809D
:10433000347F308030C20C900100E0FE900209E032
:10434000B50609E490018CF07F20801190018CE08B
:1043500004F0E0D3943240057432F0E4FFEEB4FF91
:1043600004EF4440FF223022030243EC301F0E9042
:10437000010474F0F0A3E4F0A374FB802230201356
:104380007FE01253CB90010474E0F0A3E4F0A37437
:10439000EF800C9001047480F0A3E4F0A374FBF0B0
:1043A000A374FFF0900104E0FEA3E0FF7B017A001C
:1043B00079007D047C011239EA900102E0FF640279
:1043C0006003EF70079001AFEFF08007E49001AF5A
:1043D000F0D23F900103E0FF64046003EF700690A9
:1043E00001C4EFF022E49001C4F0D23F22E4900334
:1043F000B0F0A3F0A3F09003B1E580F0A3E590F056
:10440000E49003B0F09003B0E0FFC394045055E58E
:104410009054F0FEEF44084EF590125409E5905484
:10442000F0FF9003B0E04FF5901254097580FF90B3
:1044300003B0E0FFC39402E5804010F4FE74922FB5
:10444000F582E43402F583EEF08011F4FF9003B0BE
:10445000E0248CF582E43402F583EFF09003B0E0C1
:1044600004F080A19003B1E0F580A3E0F59022C0B4
:10447000E0C0F0C083C082C0D075D000C000C001D1
:10448000C002C003C004C005C006C0079003377453
:10449000FFF0A37400F0A37422F01254313022080C
:1044A000758CE5758AF68011302108758CE0758A67
:1044B000C08006758CF0758A60900337A3E0FAA37C
:1044C000E0F91210C912542E2021033022031244A5
:1044D000EF122993D007D006D005D004D003D00224
:1044E000D001D000D0D0D082D083D0F0D0E0323014
:1044F000223ED2917580FFE52890736C93F580126F
:104500005409D290C290C2910528E528C39408406E
:1045100003E4F52830250B123F2BE52825E0243A4B
:104520008047742A2528FF123F327442252880399B
:1045300030213AD2B7D29753908F74102529F5299C
:10454000C394804003E4F529E5294290C297D2B68E
:10455000C2B6C2B70528E528C394084003E4F5288D
:10456000123F2BE52825E0243AFF123F3222E49047
:1045700003C6F0D29490028BE020E364300861908F
:1045800001FFE0FCA3E0FDA3E0FEA3E0FF90028CAE
:10459000E0F8A3E0F9A3E0FAA3E05FFFEA5EFEE93A
:1045A0005DFDE85C4D4E4F702A900203E0FCA3E0F5
:1045B000FDA3E0FEA3E0FF900290E0F8A3E0F9A3E2
:1045C000E0FAA3E05FFFEA5EFEE95DFDE85C4D4EC8
:1045D0004F600D301F089003C67480F08002C294B3
:1045E0009003C6E0FF22C0E0C0F0C083C082C0D00C
:1045F00075D000C000C001C002C003C004C005C027
:1046000006C007900335E4F0E5ACF075AC003098D7
:1046100014C2981253EF203E20E572C3941750192C
:1046200012491E8014309911C299E574C3957350D4
:1046300005123ABB8003120056900335E0F5ACD06A
:1046400007D006D005D004D003D002D001D000D0CE
:10465000D0D082D083D0F0D0E032302234E55A641A
:1046600011702EE55B64EE7028D23CD21978E07CA4
:10467000017D01FB7A00795CFE7F06120E2778E847
:104680007C017D017B007A0079627E007F0B020E47
:10469000272023033021319001A6E0FF655A7028BE
:1046A000EFF4655B7022D23CD21978F77C017D0172
:1046B000FB7A00795CFE7F06120E2778FF7C017A78
:1046C0000079627F0B123C4E22E430151790027E77
:1046D000E07011906F6693FB740193FA740293F982
:1046E0008D828032302D12906F63E493FB740193BE
:1046F000FA740293F98D82801DEF75F003A424C72C
:10470000F582E4346EF583E493FB740193FA74024A
:1047100093F9AF058F82758300120E66FEEEF4608A
:1047200012EEC39441400A9003BFE0FFEED39F40D6
:10473000027EBBAF0622203C5F9003B3E004F0E0B2
:10474000C394034002E4F09003B3E014600D1460DE
:104750001324027019E49003B5800E9003B5740120
:10476000F0E480069003B57402F0FF125391303CE0
:1047700027900372E014600D14601324027019E492
:104780009003B5800E9003B57401F0E480069003A9
:10479000B57402F0FF12539122E4789CF690026BFC
:1047A000E0FF6409704F7B017A02793CEF14FD123F
:1047B000514890026BE0243BF582E43402F583E03B
:1047C0006F7032789CF6789CE6FF243CF582E434E6
:1047D00002F583E0F4FE74252FF582E43402F583BC
:1047E000EEF006E6B408DFC21AE490037AF0C21CC9
:1047F000900373F022900373E004F022E4789CF6B7
:1048000090026BE0FD6417704F7B017A02793C12D5
:104810004D08EF4E704290023CE06421703A789C63
:10482000F6789CE6FF243FF582E43402F583E0F459
:10483000FE74252FF582E43402F583EEF006E6B42B
:1048400010DF90024FE0900235F0C21AE490037A34
:10485000F0C21C900373F022900373E004F022ABCB
:1048600007900265E054B7F9F09001AEE0FD25E055
:104870002448F582E43473F583E493FEEF5401FC9D
:10488000EE6CFEEF5402C313FCED25E02449F582E3
:10489000E43473F583E4936CFDEE33333354F84919
:1048A000FE900265F0EDC4333354C04EF0900262C6
:1048B000E0FFAE03EE1313543F4402FEEF4EF0222E
:1048C0009003C2EDF0AB07AA06E4F9D3900105E02E
:1048D0009B900104E09A500DC3900107E09B90016A
:1048E00006E09A5004E4F9803275E78175E502EA42
:1048F000F5E3EBF5E49003C2E0F5E275E64675E614
:10490000B9E4F5E553E77EAE02AF03124F6E9003B4
:10491000C2E0B5070479018002E4F9AF01229003F7
:10492000B5E01460231460332402704DE572D39413
:1049300001400AE57294145004E5996275AF72055E
:1049400072745A2FF8A69922E572D39401400CE5AF
:104950007294145006E59962758000AF7205727406
:104960005A2FF8A699E5796599FF906F6F9365774F
:10497000F579EF90706F93F57722E4FE9001DEE019
:10498000F924FEFD9001DFE0FCC39D502674D12C7C
:10499000F582E43401F583E0FC789866FF906F6F50
:1049A000937896667898F6EF90706F937896F6AE57
:1049B0000480179001DFE0FFB505067898E6FE80D9
:1049C00009E914B507047896E6FE301F038E9A2293
:1049D000AF068F9922E4789CF690026BE0FD641795
:1049E00070467B017A02793C124D08EF4E70399087
:1049F000023CE064227031789CF6789CE6FF243F0C
:104A0000F582E43402F583E0FE740E2FF582E4347F
:104A100002F583EEF006E6B411E0C21AE490037AE0
:104A2000F0C21C900373F022900373E004F022C2E2
:104A30008C438901758CDCE4F58AC28D43E780756F
:104A4000E50775E64675E6B943E20875E50675E6DD
:104A50004675E6B9D28C308DFDC28DC28C75E507E6
:104A600075E64675E6B943E20375E50675E64675F3
:104A7000E6B975E50775E64675E6B953E2FB75E5F7
:104A80000675E64675E6B9222022033021529003CE
:104A90006FE05430700F900371E0540F9073749373
:104AA0007003302A13C22CE4900369F0A3F030267F
:104AB0002FD22BD228C22622900369E475F001126E
:104AC0000F30FED3E5F09458EE9402401190036944
:104AD0007402F0A37458F0D22CD2260252D3C22C06
:104AE0002253A6BF4389109001D0E0FFE4FCFDFEF5
:104AF0007B21FAF9F8120F5C90026DE0F8A3E0F95F
:104B0000A3E0FAA3E0FB120F5C7B607AE3791678EE
:104B100000120FE7C3E49FFFE49E90039DF0A3EF14
:104B2000F090039DE0FCA3E0FDECF58DEDF58B43EB
:104B3000B708D2ABC28E22E49003C8F030230B75C5
:104B4000A01B12540975A0138013E59054F0440F74
:104B5000F590125409E59054F04407F59012540969
:104B60007580FFE580F4601690018BE004F0D3942B
:104B70000A4014740AF09003C87401F08009E490AC
:104B8000018BF09003C8F09003C8E0FF2220344866
:104B900020364520210330252190036FE0FF30E4CB
:104BA000099002C9E0B40302D234EF30E52A900242
:104BB000CFE064037022D234801E90036FE0FF3098
:104BC000E4099002CBE0B43C02D234EF30E5099026
:104BD00002E1E0B43C02D234A234E433FF22E49098
:104BE00003C1F07404F09003C1E0FF2499F582E45E
:104BF0003401F583E0F580E59054F0FEEF44084E73
:104C0000F590125409E59054F0FF9003C1E04FF580
:104C100090125409E59054F04408F5909003C1E0D7
:104C200004F0E0C3940740BE229001DFE0FFB40C23
:104C30000C789AE6301F03F59A22F59922EFD39467
:104C40000240129001DFE024D1F582E43401F583C3
:104C5000E0789A66F69001DFE024D1301F0BF582F0
:104C6000E43401F583E0F59A22F582E43401F5831A
:104C7000E0F5992275D903E4F5D87F21FEFDFC907B
:104C8000026DE0F8A3E0F9A3E0FAA3E0FB120F5CE9
:104C9000E4FB7A4BF9F8120FE7C3E49FFFE49E9020
:104CA000039FF0A3EFF090039FE0FCA3E0FDECF581
:104CB000F9EDF5E943AF0475D84043AD0422203641
:104CC00046202106302511201E0E7E007F107D001B
:104CD0007B017A0279D7802C301E0E7E007F107DFA
:104CE000007B017A0279CF801B7E007F107D007BE4
:104CF000017A0279CF1212AA7E007F107D007B011B
:104D00007A0279E71212AA2290033CEBF0A3EAF0B0
:104D1000A3E9F0A3EDF07DFF7CFF90033FE0FB14DF
:104D2000F0EB602690033CE0FBA3E475F001120F6A
:104D300046A9F0FA120E4D6CFF7E00F9906F6F934A
:104D40006DFCE990706F93FD80D0EDFEAD04EDFF3A
:104D500022C0E0C0F0C083C082C0D075D000C000C7
:104D6000C001C002C003C004C005C006C00775D89A
:104D700000D23D90026CE090026BF012282AD0071E
:104D8000D006D005D004D003D002D001D000D0D0BE
:104D9000D082D083D0F0D0E032AD07AC06D3900102
:104DA00005E09D900104E09C5013C3900107E09D35
:104DB000900106E09C4006EC54014D6004E4FF8045
:104DC0001F75E78175E503ECF5E3EDF5E475E6465F
:104DD00075E6B9E4F5E553E77EAE04AF0512517E02
:104DE00022202C4378C77C027D017B007A00792A3F
:104DF0007E007F30120E271252F2EF6008201E1143
:104E000012530F800C1231C5202A09201E031253A1
:104E10000F121A8F782A7C007D007B017A0279C7F5
:104E20007E007F30120E272213131354019003913A
:104E3000F0AF05120E4D25E04F120E93900390E057
:104E400090728793FD7004AE07801E120E4D5DFFB9
:104E50007003FE8014900390E090728793B507046E
:104E60007E018005900391E0FEAF06229003B4E03E
:104E700004F0E0C3940A4004E4F0B238302E10206D
:104E80003A0DD23AD239D238E49003B4F0C23B3072
:104E9000391C303810203B12202E06C239C23A800D
:104EA00009D2298005303B02D22BA238923B22C086
:104EB000E0C0F0C083C082C0D075D000C000C00187
:104EC000C002C003C004C005C006C007C28ED23EE7
:104ED000857271123D11D007D006D005D004D003E1
:104EE000D002D001D000D0D0D082D083D0F0D0E09A
:104EF00032125431124FABE490032FF07F487EE81A
:104F00007D01FC1232C9302318E490032FF0A31264
:104F10001098016E36007F807E257D007C00123F58
:104F2000D5120026124AE1124C7412532C02542E50
:104F3000E49003C7F012411E9003C7EFF0E0FEC0FB
:104F400006124B37D0E04F9003C7F0E0FEC00612C8
:104F500042DAD0E04FFF9003C7F09001C4E0FE902A
:104F600001AFE04E4F9003C7F0900265F022AD070D
:104F7000AC06D3900105E09D900104E09C500DC368
:104F8000900107E09D900106E09C5004E4FF801A28
:104F900075E78175E501ECF5E3EDF5E475E6467539
:104FA000E6B9AFE2E4F5E553E77E22E4F5E4AFE6E7
:104FB00075E401AEE6EF6408701BEE64F170162034
:104FC000A403D22122D22220A303D22422D225203C
:104FD000A514D21E22D223EFB40409EEB4FC05D2EC
:104FE00020024A2FD21F22E4FEFDF97C0230230268
:104FF0007C08E4FFEFC39C5027EDC39402501E745D
:105000008C2FF582E43402F583E06011F9E4FEEEC2
:10501000907364935960010D0EEEB408F20F80D4C2
:10502000AF0522E51C90736493551DFF302218EFE5
:105030006008C292C293D2928006C292C293C29278
:10504000D293C292C29322EF6008C2B5C2B4D2B565
:105050008006C2B5C2B4C2B5D2B4C2B5C2B422E4ED
:105060009003C4F07899E6301F18659AF690026CA8
:10507000E0FF04F0743C2FF582E43402F583E59AF6
:10508000F0226599F690026CE0FF04F0743C2FF575
:1050900082E43402F583E599F022900376E004F08F
:1050A000E0D3940F402E740FF0D214C215C22A7EA2
:1050B000007F137D007B017A0179F71212AA20226A
:1050C00003302110900383E0540F640260069003C4
:1050D000717408F022E49003C0F0740AF09003C0E9
:1050E000E0FF2493F582E43401F583E0F580EF449A
:1050F00018F5A01254099003C0E0F5A012540975E8
:10510000A0189003C0E004F0E0C3941340CF222025
:105110001435900377E0C394C8402C74C8F0D215BE
:10512000C22A7E007F137D007B017A0179F712127B
:10513000AA202203302110900383E0540F64026000
:10514000069003717408F02290033CEBF0A3EAF0A0
:10515000A3E9F0A3EDF0E4FFFE90033FE0FDEFC311
:105160009D501890033CE0FBA3E0FAA3E0F98F8286
:10517000758300120E666EFE0F80DEAF062290036E
:10518000B6EEF0A3EFF0E4FBFAF9099003B7E02BD9
:10519000FF9003B6E03AFE124F6EEFF46004E4F9BC
:1051A000800D0BBB00010AE4B503E0EAB402DCAFFA
:1051B0000122E4FFFEFDFCEDC39402501E74252F76
:1051C000F582E43402F583E06011FCE4FEEE9073B6
:1051D00064935C60010D0EEEB408F20FEFB408D7D3
:1051E000AF0522E4FFEF25E0246FF582E43471F58A
:1051F00083E493FC740193FDEF25E0240AF8A604F0
:1052000008A6050FEFB408DD22E4FF900289E02034
:10521000E3193008169001FFE0FCA3E0FD90028C3A
:10522000E05CFCA3E05D4C60027F802290037AE0AA
:1052300004F0E0D3940F4016740FF0D21AC21C7E13
:10524000007F087D007B017A0279251212AA229044
:105250000383E0540FFF6408600EEF640E600920C2
:105260001406201503302D03C23722D237D22BD299
:10527000282220230330211A30230790028BE030AC
:10528000E50A30210A900289E020E5031212D612C5
:10529000542522201A1D900373E0C394C84014744F
:1052A000C8F0D21C7E007F087D007B017A02792540
:1052B0001212AA222021033025067E007F208007BB
:1052C00030240F7E007F307DFF7B007A00792A1228
:1052D00012AA222021033025067E007F208007307D
:1052E000240F7E007F307D007B007A00792A121225
:1052F000AA22E4FF30371790037BE0D3943C4006AA
:10530000E4F0C237800890037BE004F07F01223094
:105310002805C22802359990036FE030E608124B49
:105320008DEF70078002C234122C3A2212436612AB
:1053300051E312001E9003BF74E9F09003BE745F46
:10534000F09002647401F02220220330210C12003C
:10535000661230BA124E6C124DE1302303122AEE5F
:1053600022301F03B29022302003B2EA2230210300
:10537000B2B322302202B294229001F7E0540FFE21
:10538000600864016004EEB40904E4FF80027F2039
:1053900022E4AEACF5ACEF60057598D0800375984B
:1053A00050AF068FAC22124A8812509A12510F3019
:1053B000230612522C1252932290039FE0FCA3E08A
:1053C000FDECF5F9EDF5E975D840228FE275E504BD
:1053D00075E78175E64675E6B953E77F2220180523
:1053E000124C29800312497A9001DFE004F02290E8
:1053F000039DE0FCA3E0FDECF58DEDF58BD28E2254
:10540000302303C2B522C2B222E4FF000FEFB4057D
:10541000FA2212540943E110221247360253A6120F
:10542000536102267E12170B023B8A0200FED2AFA6
:1054300022C2AF2222000000000000000000000095
:10544000000000000000000000000000000000005C
:1054500000000000000000000063949010214080D4
:1054600084F3DE0909098E4949499E2364242020DA
:1054700021222477844A5151911F1111D19E49490B
:10548000498E090909DE2364202021202024738409
:105490004A5151915F5151919F49484A8E4A48481B
:1054A0009CDE4949890E0909091E000000003C3CA8
:1054B000000000276420202121212171C44A51913C
:1054C000111F1111113E63676F7B7363633E1838C0
:1054D0007818181818187E3E6303060C1830637F7E
:1054E0003E6303031E0303633E060E1E36667F06FD
:1054F000060F7F6060607E0303633E1C3060607E49
:105500006363633E7F6303060C181818183E6363D9
:10551000633E6363633E3E6363633F0303063C3362
:105520004A4A0A11204042799E494949CE4949498F
:105530009E276424242320202473C40A1111915F20
:10554000515191236424242320202473844A5151EF
:10555000D15F515191060E0606E6E606060F081CBD
:105560003663637F6363637E3333333E3333337E2B
:105570001E336160606061331E7C363333333333F6
:10558000367E7F3331343C3431337F7F3331343CAA
:10559000343030781E336160606F63331D63636342
:1055A000637F636363633C181818181818183C0F5E
:1055B000060606060666663C733336363C363633D8
:1055C0007378303030303031337F63777F6B636393
:1055D00063636363737B7F6F676363631C366363BB
:1055E000636363361C7E3333333E303030783E6342
:1055F0006363636B6F3E067E3333333E3633337300
:105600003E6363301C0663633EFF99181818181830
:10561000183C63636363636363633E6363636363F1
:10562000631C080063636363636B7F773663636344
:10563000361C36636363636363361C1C1C1C3E7F2D
:1056400063460C182061637F2364242427242424C8
:1056500073844A1111915F515191183C7EDB1818E7
:105660001818181818181818DB7E3C189E49494954
:105670008E4949499E000000000000000000000023
:10568000000000000000000000000000000000001A
:10569000000000000063941023408084F3BC1212C9
:1056A0001C9292923C47C84041424448EF0894A261
:1056B000223E2222A23C92921C121212BC47C840E7
:1056C00043404048E70894A222BEA2A2223EA0A0E6
:1056D00020BCA0A020BC92921C1212123C00000020
:1056E0003E000000004FC84041424242E28894A27E
:1056F000223E22222238444444444444381030108C
:105700001010101038384404081020407C3844042D
:10571000180404443808182828487C08087C4040AD
:10572000380404443838444078444444387C4404C1
:105730000810101010384444384444443838444465
:10574000443C04443867941423408084F33C929290
:105750009C9292923C4FC84847404048E7881422A8
:1057600022BEA2A22247C84848474048E70894A260
:10577000A2BEA2A222040C0404E404040E102844D5
:10578000447C4444447824243824242478384440F5
:10579000404040443870484444444448707C404051
:1057A000784040407C7C4040784040404038444015
:1057B000405C4444384444447C44444444381010DD
:1057C00010101010381C08080808084830444850C9
:1057D0006060504844702020202020247C446C6C61
:1057E000545454545444646454544C4C44384444C5
:1057F00044444444387824242438202070384444D5
:10580000445454380C784444784844444438444020
:1058100030180444387C1010101010101044444408
:105820004444444438444444444428381044545480
:1058300054547C3828444428101028444444444498
:1058400028101010107C0408101020407C46C94815
:105850004E494949E6102844447C44444410385495
:10586000101010000010101054381000003C9292DC
:105870001C9292923C0000030007800CC01860301C
:1058800030303030303FF030303030303030303049
:10589000307878000000003FC018601830183018C9
:1058A0003018601FC01860183018301830183018C1
:1058B000603FC00000000007E00C7018303000307E
:1058C0000030003000300030003000300018300C64
:1058D0007007E0000000003F8018C0186018301802
:1058E0003018301830183018301830183018601848
:1058F000C03F80000000003FF0183018101800185A
:105900000018C01FC018C018001800180018101880
:10591000303FF0000000003FF01830181018001859
:105920000018C01FC018C018001800180018001870
:10593000003C000000000007C00CE0186030603040
:105940000030003000300030F03060306018600C03
:105950006007C0000000003CF01860186018601874
:105960006018601FE01860186018601860186018F0
:10597000603CF0000000000FC003000300030003C0
:1059800000030003000300030003000300030003FF
:10599000000FC00000000007E001800180018001CD
:1059A000800180018001800180018001803180338D
:1059B000001E00000000003CE0186018C0198019AB
:1059C000801B001E001B001980198018C018C01809
:1059D000603CF0000000003C00180018001800189F
:1059E00000180018001800180018001800181018E7
:1059F000303FF000000000303038703CF037B033FA
:105A00003033303030303030303030303030303093
:105A1000303030000000003030383038303430342E
:105A200030323033303330313030B030B03070302D
:105A30007030300000000007800CC018603030303B
:105A40003030303030303030303030303018600C62
:105A5000C00780000000003FC018601830183018E0
:105A60003018601FC018001800180018001800181F
:105A7000003C000000000007800CC018603030308F
:105A800030303030303030363033301B600FC003B0
:105A9000E000F0000000003F8018C0186018601897
:105AA000C019801F001B001980198018C018C01869
:105AB000603CF0000000000FC018E03060300030A3
:105AC0000018000E00038000C00060003030303845
:105AD000601FC0000000003FF033302310030003BC
:105AE000000300030003000300030003000300039E
:105AF000000780000000003CF01860186018601873
:105B00006018601860186018601860186018600CE1
:105B1000C00780000000003CF01860186018601892
:105B2000601860186018601860186018600CC00772
:105B30008003000000000030303030303030303032
:105B4000303030303030303330333037B03CF038F4
:105B5000703030000000003CF018600CC00CC00732
:105B600080078003000300078007800CC00CC0186A
:105B7000603CF0000000003CF018601860186018ED
:105B8000600CC00780030003000300030003000350
:105B9000000780000000003FF03030206000C000AF
:105BA000C001800300030006000C000C0018103038
:105BB000303FF00000000000000000000000000086
:105BC0000000000000000000000000300030001065
:105BD000002000000021102110391027FC4110790D
:105BE00010AFFE2000FBF82208220823F82A083212
:105BF0000823F80208000043F82208220803F800EE
:105C000000E00027FC204020402FFE204020A03153
:105C10001022080C0610481048284825FE4248BCAF
:105C20004811FE1000FEFC1084948458FC50841E21
:105C300084F0FC4084200011FC0104FD0401FC7888
:105C400000000079FC002078204BFE482048507866
:105C50008849040202100010F81088FE881088108D
:105C60008838883488548850889108110A120A129A
:105C70000A140600001210121022102FFC6210A24B
:105C80001022103FFE200022102208240C2804209D
:105C90000000000000020001043FFE20702F802859
:105CA0008028882FFC288028404A405C24881407DC
:105CB000CC000000001080104417FEFC00101011F2
:105CC000F8111011101D10F11041100212021204EF
:105CD0000E0000000001104110211037FC211001BE
:105CE000100110F7FE1110111012101210141028CC
:105CF0000047FE000002002240223022107FFE24D6
:105D000000040007E00C200A200A201140208041F6
:105D100060861C180801000100010801187D20059B
:105D2000C0058009601110210E41048100050002A8
:105D3000000000000008080BFC0A081208120833D3
:105D4000F8324050449FFE104010E01150124814A9
:105D50004610C00000044002807FFC01003FF801B3
:105D600000FFFE04400830344EC4440440044008A0
:105D700040104000000100010001047FFE41044189
:105D80000441047FFC410401000100010001000105
:105D90000001000000412031241FFE012080006F1F
:105DA000FC212001201FFC2924E9242AD42C0C28C2
:105DB000142808000008507F4808480840FFFE10DB
:105DC00040FF40204828487E3008200F60F89209A4
:105DD0000A0A060000040025F8251024A024402407
:105DE000B0070E04041FC0010006103FF80108119F
:105DF000102308000007E0084000887FFC0008002E
:105E0000081FF8000800087FF8020851045112909A
:105E1000120FF00000001043F830001000000807D7
:105E2000FCF080108011001120121017F8100828C3
:105E30000047FE000010401048FDFC204028444B65
:105E4000FE7C80088009FC1C08E810489008600867
:105E50002008100000010001103FF802000204FFBA
:105E6000FE040004100FF80010002000400680011E
:105E7000800040000000083FFC2108210821083F65
:105E8000F82108210821083FF8210821084108418C
:105E900028801000000200020002107FF842104229
:105EA000107FF0421042107FF04210020402040200
:105EB0000401FC0000111010A013F8FC4810483336
:105EC000F83A40564453FE90C411441254144818F2
:105ED0004010400000104010401044FEFE11081217
:105EE0008810887C8844884450442044207C504456
:105EF0008E0304000000407BF8491050A057FE605C
:105F00000053F84A084BF84A086BF850404FFE40DF
:105F100040404000003EFC2288228822883EB02279
:105F20008022FC22A43EA422A8229022A822A84AD1
:105F3000C684840000080008200FF0182026C04105
:105F40000006C00A30320EDFF402100410041008FC
:105F5000A0304000000010403833C010400044F72B
:105F6000FE10401040104813FC120816081A0813BF
:105F7000F8020800000100010001001108111811C9
:105F8000202140428002800440044008201010205C
:105F90000E40040000020001007FFE400281041157
:105FA0001011181120214002800280044008301096
:105FB0000E600400000E20792208A408A87DFC19B8
:105FC000041D042BFC2904490449FC890409040923
:105FD000140908000010001BF8101027FE290069A2
:105FE00000A9FC29402A402FFE28A0289021182231
:105FF0000E2404000000404248315011608040638C
:10600000F822080A0813F82208E20823F8220822D6
:10601000282210000000807C40444048044FFE507D
:1060200080488848FC448844886888510841084270
:1060300050442000000040204022402240224822BC
:106040007CFBC8264822482248226822503A42E275
:106050000241FE00001FF001007FFE51128D64110D
:10606000103FF820002FF020003FFC2A1029204884
:10607000C08C38000000010002000400080010007D
:1060800020004000800100020004000800100020F1
:106090000040008000000000000000000000000040
:1060A00000000000000000000000000000000000F0
:1060B000000000000020001BF81048FC4800487C4D
:1060C0004801F87C4800487C484448444A444A7C9B
:1060D0004644420000A204C47EF740A240D540FFDF
:1060E0007E8048FF48A248C448F748A248F7489134
:1060F00088FF8801081FF8100010001FF010001F13
:10610000F01000FFFE14001210112010C012201415
:1061100018180E100400000000000000000000002D
:10612000000000000000000000000000000000006F
:10613000000000000000000000000000000000005F
:10614000000000000000000000000000000000004F
:1061500000000000007EFC42847EFC42847EFC4005
:10616000044FE4444444445FF444444844484450A5
:10617000444014400800000000000000000000003F
:106180000004000300038001C000C0000000000004
:1061900000000000000000000000000000000007F8
:1061A0008008400840084007800000000000000010
:1061B00000000000000000000000000000000000DF
:1061C000000000000007C01FF03838600C40048059
:1061D00002000000000000000080024004600C3853
:1061E000381FF007C00000000000000000000000A1
:1061F000000000000003800D601110254828284889
:1062000024501450144824282826C811100D600169
:10621000000000000000000000000000000000007E
:1062200000018003C00180000000000000000000A9
:106230000000000000020001001F00010801187D9D
:10624000A005C0054009201110210E4104050002DF
:1062500000000000000100010001000104FFFE0138
:1062600000010002800240044004200810100E606B
:1062700004000000002148224824D0277CFA482549
:106280005427FC204477FEAA442228251028AA205F
:106290004600000000FFFE01007FFE51128924111C
:1062A0001001003FF821083FF821083FF8010000E5
:1062B000FC000000000040804047FC2040F7FC1438
:1062C0004427FC444427FC20402FFE30404C4083B0
:1062D000FE00000000208020FC40848988FA5010D5
:1062E0002020504888FB0621FEA904A904A9FC210E
:1062F000040000000008207FFC01007FFC0100FF7B
:10630000FE0BA01FF029284FE4891208A009400CB9
:10631000380000000000803FFE00801FFC10841F3A
:10632000FC10841FFC00127FFE00100310011000FF
:1063300050002000000100110011083FFC21004125
:1063400000810001103FF80100010001000104FF7D
:10635000FE00000000020001007FFE4002802400D9
:10636000247FFE0020082004200420002000A0003C
:106370004000000000411061102FFE11100110615B
:10638000F0204017FC0554055416EC2444645424B2
:10639000480000000008503E480848FFFE08403E04
:1063A0004008403E482A483E302A203F6008927FFD
:1063B0000A08060000824044204FFC1420E42027F5
:1063C000FC4420C42027FC2420242027FC54008FD8
:1063D000FE000000000040F88411FE66882050FC9A
:1063E000202B8E20206020A3FC20442084210466E2
:1063F00038000000002008101CFDE0002078200379
:10640000FE7820002079FC49044904490479FC49BC
:1064100004000000007EFC48847E4842307E6848CC
:10642000867F0204401F8002203FF00920111021C6
:106430000800000000108421084210210810840187
:10644000004104210819300100028004401830E0A6
:106450000E000000000100FFFE01003FF821083F90
:10646000F801003FF80108FFFE01083FF8010007AE
:1064700000000000000200040008083FFC20082083
:10648000083FF8200820083FF8200820083FF8209F
:10649000080000000001007FFE400280043FF01A67
:1064A0001063300540198063400530190E65040201
:1064B000000000000000203FC011100D300544FF17
:1064C000FE092011103FFED1141FF011101FF01013
:1064D0001000000000F82088388820FBFE0222020D
:1064E000FCFA20223C42007A480A480A48924A6450
:1064F0008E000000007CFC0440482E30102EF84234
:106500009482923E9C20003EF80288025022201C79
:10651000D8000000008FFE484207FCF04017FC2422
:106520004447FC844447FC20402FFE204050408FCD
:10653000FE000000002020FBFE2020F9FCA9F4A9A9
:1065400024F9FCA822ABFEF80821FEF808208820D8
:106550001000000000104010441FFE204067FCA403
:1065600044244427FC2244218020C02130260E28C8
:106570000400000000004047FC304023F8004007C2
:10658000FEF00013F8120813F8120813F816081A90
:10659000281210000000204F10297C29480F2808DD
:1065A00010E8FE2F102D102D7C35102710201050D4
:1065B000008FFE000000A00090F91009FE8B204B18
:1065C000202DFC1120192029FC25204520812001A7
:1065D000FE0100000000000000000007C00C600C7D
:1065E000E00DE00F600E600C600C6007C000000062
:1065F0000000000000000000000000018003800790
:10660000800180018001800180018007E00000009E
:10661000000000000000000000000007C00C600047
:106620006000C00180030006000C600FE000000065
:10663000000000000000000000000007C00C600027
:1066400060006003C0006000600C6007C0000000D4
:10665000000000000000000000000000C001C003B6
:10666000C006C00CC00FE000C000C001E000000088
:1066700000000000000000000000000FE00C000C13
:10668000000C000FC0006000600C6007C00000003C
:106690000000000000000000000000038006000C65
:1066A000000C000FC00C600C600C6007C000000004
:1066B00000000000000000000000000FE00C60007F
:1066C0006000C0018003000300030003000000001D
:1066D000000000000000000000000007C00C600C7B
:1066E000600C6007C00C600C600C6007C00000000C
:1066F000000000000000000000000007C00C600C5B
:10670000600C6007E00060006000C00780000000CF
:106710000000000000202013FEFC2001FC78200374
:10672000FE000079FC010479FC490449FC49047924
:10673000144908000000204F10297C29480F280820
:1067400010E8FE2F102D102D7C3510271020105032
:10675000008FFE00002440FF5024483CFE08C87F04
:10676000484A7E7E4808487E7E0848FF48144822F2
:106770007EC040000008400C200BFE100011F831D4
:106780000851F8900017FE140211FC102010201080
:10679000A0104000000000F81C13E0102020207919
:1067A00020293C09204920492029FE1000280046C4
:1067B0000081FE000000000000000000000000005A
:1067C00000000000000000000000000000000000C9
:1067D0000000000000020002000200FFFE020002B2
:1067E0000007F004100620092008C010C021204234
:1067F000188C0E30042040204027FC3040ABF8A01D
:1068000040AFFE200023F8220823F8220823F822B4
:106810000822282010100011F81108FDF8110811A5
:10682000F8180037FC50409240127C124016401578
:10683000C0587E200000001FF80000000000007F0C
:10684000FE01000100112011102108410C810401FA
:106850000005000200010001000100FFFE038003AB
:106860004005400520091011182FEEC10401000158
:10687000000100000000003FF00010001000102098
:10688000103FF02000200020002004200420063FBC
:10689000FC0000000020403F7E48504488891008DA
:1068A0001017FE101032105110919010901010100F
:1068B0001010501020010002800440082010182001
:1068C0002EDFF4000000001FF01010101010101F39
:1068D000F010100000040004000FF0102020405FB2
:1068E000F8110811081FF812480240044004420839
:1068F00042103E200002403FF802483FF822403F4D
:10690000FE0442084A1FF468100910091009100219
:10691000C00C3830101040104010A0FD10120E387E
:106920000035F850005088924C1148115010201733
:10693000FE100000000100010001007FFE0540097B
:1069400030310EDFF410101FF0101010101FF00087
:10695000007FFE00001080108020807CFC450445F4
:106960000446047C8444444464442444047C044435
:106970002840100000040004000FF00C20124061B9
:106980008002600D1E71081FFC01000920111821F2
:10699000080500020010401A401340324023FC64F6
:1069A00040A44028402FFE2040204020402040208E
:1069B0004020402040FFFFFFFFFFFFFFFFFFFFFFE2
:1069C000FFFFFFFFFFFFFFFFFFFFFFFFFFFFFFFFD7
:1069D000FFFFFFFFFF400027F82090006007F8044A
:1069E00048E7F82448244827F824482468245050CD
:1069F000008FFE0000400027F8310821080108F14F
:106A00000817E81108110811081108110A150A19C8
:106A10000A110400000400440E65705540564044BD
:106A2000407F7E4C48564855486448448844887F97
:106A3000080208000810401020102013FEFE041069
:106A40004014401BFE10883110D190106010581176
:106A50008E56042000044004407FFC04400440FFA4
:106A6000FE01001FF011101FF0111011101FF0088F
:106A700020101860080400040007F0082010403FB0
:106A8000F05110111011101FF0100010041004101C
:106A9000040FFC0000080008FC10241F2420243EE2
:106AA00024482408FC7E440844084408440A440C52
:106AB0004409FE00000040005000487FFC004000F8
:106AC000403E40224C22483E30002002540C947339
:106AD0000C0C040000204022482244FA4023FE20EF
:106AE00040208028F83088E150215022202450296D
:106AF00088A60640001000100013FE1020FE201093
:106B000020142018203020D0201020102010201019
:106B10002050A02040020002007FFE040004000874
:106B200040084017FC304050409040104010401743
:106B3000FE1000000010000BFC08042004200420BC
:106B40000420042004200420042004200420042025
:106B5000042014200800007FFE04200420042004E8
:106B600020FFFE04200420042008200820102020FC
:106B70002040200000003E0FC0080008000FFE0863
:106B800000080008000BFC12041204120423FC226B
:106B90000442040000020001047FFE066011881216
:106BA0004814281FF801003FFC244428242FF42017
:106BB0001420142008000027F011101110011001FA
:106BC0001077D011101112110A110A1106110228A2
:106BD0000047FE00000040604017FC104003F80230
:106BE00048F24813F810E01150124814441040685D
:106BF0000047FE000020801040104007FE80404803
:106C0000404840104013FC2040E0402040204020FD
:106C1000402FFE200001003FFC08200440FFFE0042
:106C2000001FF0121011101FF000002908288468BE
:106C30001407F000000080008000800080088008B9
:106C40008008FC0880088008800880088008800888
:106C500080FFFE000008200430062004487FFC016D
:106C60000001000100FFFE01000280044008201026
:106C700030201C4008003CFBC088488A4C89488969
:106C80005088408BFEF840884000400040004001A2
:106C9000400080000000047C844484448444844494
:106CA00084449C7DE4448440040004000400040007
:106CB00004000400003E7C224422443E7C22443EE8
:106CC0007C2004200420042004200420042004202C
:106CD000042014200808400C60108821F048400C63
:106CE0008819FC3008510091F813101490186010A6
:106CF00090110E160410100848FF48287E52D06BE1
:106D0000507E7C0850FF509150957CBF508150813F
:106D100050857E82403FF821083FF821083FF8085F
:106D20002008207FFC08200820FFFE00000820101B
:106D300010200800000100111009207FFE40029F72
:106D4000F410101FF001003FF8210821082128212C
:106D500010010001007E7C42447E7C42447E7C40E7
:106D60000444444A945CE44A545EF4448454A45C6D
:106D7000E44884508C080009FC08447E4408440818
:106D800094FF0808FC288428842E8428FC280058B6
:106D9000004FFE8000676869FF727374755BA9CF4E
:106DA000D0D1CFD2D3D4D57278B0ACACB4AEACAE77
:106DB000ADB2B4FF7F80A9AAABFF797AA9AAABFFD5
:106DC0007D7E6E6FFFCCCD69CEFFE96BFFB9725B44
:106DD000A9D6D7D8D9DAD8FFB9DF76775BD7D8D993
:106DE000A9DBDCDAD8FF6572606172FF62636466FA
:106DF000FFBBBBFFDDDEB9DFD8E0FF679569FF743D
:106E000075B6CF9E6DE1E2CFD2FF7F80B6B7B8FFF7
:106E1000799FB6B7B8FF7D7EA6A7FFCC836984FFB4
:106E2000E99AFFB9925BB6D6E388E4E588FF9273EE
:106E3000E6E75BE388E4B6E588FFA592916192FFFF
:106E400062639B66FFDDDEB9DF88E8FF4D41494E96
:106E50005441494EFF4552524F52FF45415254480A
:106E60005155414B45FF46495245FF464952454D14
:106E7000414EFF4552524F52FF4F564552BB4C4F69
:106E80004144FF504F574552BB435554FF5741496A
:106E900054FF47454E455241544F52FF57415445C8
:106EA00052FF53544F50FFBBBBBBBBFFCCCD5C5D0F
:106EB000FFCC835E5FFF434F4DBB455252FF4F50A7
:106EC000424144AE5245FFFF6EA7FF6EA7FF6D958E
:106ED000FF6D99FF6DB4FF6DBAFF6DC0FF6EA7FF28
:106EE0006DC5FF6DCAFF6DCDFF6DD8FF6DE6FF6DFF
:106EF000ECFF6DF1FF6DF4FF6EA7FF6EA7FF6DFB5A
:106F0000FF6DFFFF6E0AFF6E10FF6E16FF6EA7FF8C
:106F10006E1BFF6E20FF6E23FF6E2EFF6E3AFF6E1C
:106F200040FF6DF1FF6E45FF6EA7FF6EA7FF6E4C31
:106F3000FF6E55FF6E5BFF6E66FF6E6BFF6EA7FF09
:106F40006E73FF6E79FF6E83FF6E8DFF6E92FF6E24
:106F50009CFF6DF1FF6EA2FF6EA7FF6EA7FF6EA7ED
:106F6000FF6EA7FF6EBEFF6EACFF6EB1FF6EB60088
:106F7000C1814001C0804101C0804100C181400108
:106F8000C0804100C1814000C1814001C0804101F9
:106F9000C0804100C1814000C1814001C0804100EA
:106FA000C1814001C0804101C0804100C1814001D8
:106FB000C0804100C1814000C1814001C0804100CA
:106FC000C1814001C0804101C0804100C1814000B9
:106FD000C1814001C0804101C0804100C1814001A8
:106FE000C0804100C1814000C1814001C080410199
:106FF000C0804100C1814000C1814001C08041008A
:10700000C1814001C0804101C0804100C181400078
:10701000C1814001C0804101C0804100C181400167
:10702000C0804100C1814000C1814001C080410059
:10703000C1814001C0804101C0804100C181400147
:10704000C0804100C1814000C1814001C080410138
:10705000C0804100C1814000C1814001C080410029
:10706000C1814001C0804101C0804100C181400018
:10707000C0C101C30302C2C60607C705C5C404CC0C
:107080000C0DCD0FCFCE0E0ACACB0BC90908C8D83C
:107090001819D91BDBDA1A1EDEDF1FDD1D1CDC14FC
:1070A000D4D515D71716D6D21213D311D1D010F0CC
:1070B0003031F133F3F23236F6F737F53534F43C4C
:1070C000FCFD3DFF3F3EFEFA3A3BFB39F9F838281C
:1070D000E8E929EB2B2AEAEE2E2FEF2DEDEC2CE43C
:1070E0002425E527E7E62622E2E323E12120E0A0AC
:1070F0006061A163A3A26266A6A767A56564A46C8C
:10710000ACAD6DAF6F6EAEAA6A6BAB69A9A86878BB
:10711000B8B979BB7B7ABABE7E7FBF7DBDBC7CB47B
:107120007475B577B7B67672B2B373B17170B0508B
:107130009091519353529296565797559594549CCB
:107140005C5D9D5F9F9E5E5A9A9B5B99595898889B
:107150004849894B8B8A4A4E8E8F4F8D4D4C8C44BB
:10716000848545874746868242438341818040002B
:107170001400190032006400FA01F403E805DC0190
:1071800002040810204080090102010301020104E9
:1071900001020103010201050102010301020104D0
:1071A00001020103010201060102010301020104BF
:1071B00001020103010201050102010301020104B0
:1071C000010201030102010701020103010201049E
:1071D0000102010301020105010201030102010490
:1071E000010201030102010601020103010201047F
:1071F0000102010301020105010201030102010470
:10720000010201030102010801020103010201045C
:10721000010201030102010501020103010201044F
:10722000010201030102010601020103010201043E
:10723000010201030102010501020103010201042F
:10724000010201030102010701020103010201041D
:10725000010201030102010501020103010201040F
:1072600001020103010201060102010301020104FE
:1072700001020103010201050102010301020104EF
:1072800001020103010201000103070F1F3F7FFFFD
:1072900001010101010101010101010101010101DE
:1072A00001010101010101010101000001010101D0
:1072B00000000101000000000000000100000000CB
:1072C00001010101010101010000000000000000B6
:1072D00000000000000000000101000001010101A8
:1072E000000001010000000000000001000000009B
:1072F000000000000000000002020202020202027E
:10730000020202020202020200000000000000006D
:10731000000000000000000000000000000000006D
:107320000102FB0102FE0102FF0102FA0102FC015F
:1073300002FD4F504241443152460000000000001F
:10734000010204081020408000000001010001013A
:10735000000000000000000000000000000000002D
:10736000000000000102040810204080FEFDFBF731
:10737000EFDFBF7F000001010101010001010101F8
:047380000101010105
:00000001FF
